:100000000C94AC020C94C7020C94C7020C94C70267
:100010000C94C7020C94C7020C94C7020C94C7023C
:100020000C94C7020C9462130C94C7020C943F13F7
:100030000C9468200C94C7020C94C7020C94C7025D
:100040000C94C7020C94C7020C94E8110C94C702DC
:100050000C94B2060C94C7020C9477060C94C70259
:100060000C9490150C94C7020C94461F0C94C70274
:100070000C94C25D0C94C7020C94C702A71FBA1F50
:10008000AE1FF81F0820EA1FD61F871F761F042007
:10009000A21F6D1F7A1F761FF41FFF1F6D1F7A1F8F
:1000A000761F1C2017206D1F961F0A0D466C69676E
:1000B0006874436F6E74726F6C0A0D486172647776
:1000C0006172653A25642E25640A0D536F66747754
:1000D0006172653A5625642E2564256320000A0D59
:1000E0003D3D3D3D3D3D3D3D3D3D3D3D3D3D3D3D40
:1000F0003D3D3D3D3D3D3D3D3D3D3D3D3D3D000AA0
:100100000D496E69742E20454550524F4D3A204797
:10011000656E65726174696E672044656661756CB1
:10012000742D506172616D6574657220616E64201A
:10013000537469636B2D53657474696E67732E2EE7
:100140002E000A0D496E69742E20454550524F4DC0
:100150003A2047656E65726174696E672044656612
:1001600061756C742D506172616D65746572207576
:1001700073696E67206F6C6420537469636B2053DE
:10018000657474696E6773000A0D414343206E699C
:100190006368742061626765676C696368656E2176
:1001A000000A0D42656E75747A6520506172616D4A
:1001B000657465727361747A202564000A0D557345
:1001C000696E67202573000A0D4162676C6569637B
:1001D00068204C756674647275636B73656E736FBB
:1001E000722E2E000A0D4F4B0A0D000A0D53746536
:1001F000756572756E673A200048656164696E675F
:10020000486F6C64004E65757472616C000A0A0D6B
:10021000002E005B25695D005B25695D002B204D8C
:10022000696B726F4B6F70746572202B0048573A80
:100230005625642E25642053573A25642E256425BF
:10024000630053657474696E673A20256420002842
:10025000632920486F6C676572204275737300488C
:100260006F6568653A202020202025356900536F8E
:100270006C6C486F6568653A20253569004C756679
:1002800074647275636B3A20253569004F66662089
:1002900020202020203A20253569004B65696E65B5
:1002A000200048F668656E726567656C756E67005C
:1002B000616B742E204C616765004E69636B3A2058
:1002C000202020202025356900526F6C6C3A2020B8
:1002D00020202020253569004B6F6D706173733AC3
:1002E000202020253569004B313A25346920204BE8
:1002F000323A25346920004B333A25346920204BAB
:10030000343A25346920004B353A25346920204B96
:10031000363A25346920004B373A25346920204B82
:10032000383A25346920004E693A25346920205234
:100330006F3A253469200047733A253469202047F5
:10034000693A253469200050313A2534692020501B
:10035000323A253469200050333A25346920205040
:10036000343A25346920004779726F202D20536577
:100370006E736F72004E69636B20253469202825E7
:1003800033692900526F6C6C20253469202825338D
:100390006929004769657220253469202825336959
:1003A00029004E69636B202534692028253369298B
:1003B00000526F6C6C202534692028253369290090
:1003C0004769657220253469202825336929004E44
:1003D00069636B2025346920282533692928253352
:1003E000692900526F6C6C202534692028253369F7
:1003F0002928253369290047696572202534692039
:100400002825336929282533692900414343202DB4
:100410002053656E736F72004E69636B20253469DB
:1004200020282533692900526F6C6C2025346920FF
:10043000282533692900486F6368202534692028FE
:1004400025336929005370616E6E756E673A2020FE
:1004500025356900456D70662E506567656C3A25D7
:100460003569004B6F6D7061737320202020202050
:1004700020005269636874756E673A2020253569DB
:10048000004D657373776572743A202025356900D5
:1004900053746172743A2020202020253569005061
:1004A0006F7469313A202025336900506F746932C6
:1004B0003A202025336900506F7469333A20202593
:1004C000336900506F7469343A2020253369005332
:1004D0006572766F202000536574706F696E7420AA
:1004E00020253369005374656C6C756E673A20255E
:1004F00033690052616E67653A2533692D2533698A
:100500000045787465726E436F6E74726F6C202054
:10051000004E693A2534692020526F3A253469200B
:100520000047733A253469202047693A2534692009
:100530000048693A253469202043663A2534692009
:10054000000A0D55415254203120696E6974696169
:100550006C697A65642E000011241FBECFEFD0E1D4
:10056000DEBFCDBF13E0A0E0B1E0E4E4F1EC02C0F7
:1005700005900D92A03CB107D9F718E0A0ECB3E0CC
:1005800001C01D92A53AB107E1F70C9469030C94E0
:100590000000282FFB018150853008F023E0842FD4
:1005A0009927332721503040829FD001839FB00D7F
:1005B000929FB00D1124AC59BF4F019724F00E94B7
:1005C00084600192FACF0E944A5A0895863038F02A
:1005D00085E0A2E0B0E0082E0E9491600895882393
:1005E000C1F70895582FFB01863010F155E0842F94
:1005F0009927252F332721503040829FD001839F98
:10060000B00D929FB00D1124AC59BF4F019724F04B
:1006100001900E949160FACF852F563060F085E0FE
:10062000A2E0B0E0082E0E9491600E944A5A08950C
:100630008823E9F3DCCF552399F70E944A5AF7CF74
:1006400022E030E0D9010E948460802D982F8150F3
:10065000853028F093E0D901092E0E949160892FFE
:100660009927089520919407E22FFF27EE0FFF1F8F
:10067000EA59F84F808191818D5E9F4F14F010925E
:100680000201408151814A5B5F4F24F430910201A5
:10069000332319F02091630615C051E050930201F5
:1006A00020916306250F20936306253038F068EE0D
:1006B00073E07093E0036093DF0304C0822F0E9415
:1006C0006023E8CFA22FBB27B0933107A093300758
:1006D0000895CFEFD0E1DEBFCDBF14B815B887EED7
:1006E00093E0C29797FFFDCFC8EED3E0189BF3C20B
:1006F000199BEFC22DE02093010191E897B93E9A32
:100700007FEF78B96BE164B951E055B94EE34AB96E
:10071000579A37E73BB914B7177F14BF00916000B1
:100720000861009360001092600080ED97E0909364
:10073000E0038093DF031092400410923F04109274
:100740006B0710926A0710924204109241041092B3
:100750004404109243042A3009F4B9C2243109F444
:10076000B6C2289A0E94DB120E94D60B0E947A140D
:100770000E94051F0E94C15678944BE650E05F939B
:100780004F9307E410E01F930F931F921F928091E5
:1007900001016AE00E941460A92EBB24BF92AF92AF
:1007A000809101010E94146099279F938F938AEA98
:1007B00090E09F938F931F920E94990EEDB7FEB722
:1007C0003D960FB6F894FEBF0FBEEDBFAEEDB0E0A4
:1007D000BF93AF931F920E94990E209101010F9039
:1007E0000F900F902C3008F070C2299AE4E9F7E0DE
:1007F00039E006E710E0D801132E0E948C600E94B9
:100800004A5A05571040D8010E948460F02DFF3FDE
:10081000B9F0D8010E948460502D593488F0B0910D
:100820009407BA3068F4609195076A3048F4709183
:1008300096077A3028F4909197079A3008F4FFC110
:100840002FEF30E03F932F931F920E94990E0E944A
:100850005F210F900F900F90D8010E948460F02DBF
:10086000F93409F09FC182E0E82E80E0F82EA4E080
:10087000B0E00E948460102D153008F0F2C1D7015D
:100880000E948460202D922F2150253028F093E083
:10089000D701092E0E949160E4E9F7E046E5392F7F
:1008A0003150353008F093E0892F9927019766E59C
:1008B00070E0869FD001879FB00D969FB00D1124E8
:1008C000AC59BF4F142E0E948C600E944A5AD70127
:1008D0000E948460402D942F4150453028F093E0D1
:1008E000D701092E0E949160E92EFF24FF92EF921A
:1008F000E1EAF1E0FF93EF931F920E94990EB0900E
:10090000C7070F900F900F900F900F90B2FEA6C1E7
:100910000E94135CD090C707D2FED4C183E091E05F
:100920009F938F930CEB11E01F930F931F920E94E4
:10093000990EF0909C070F900F900F900F900F90D2
:10094000F0FC9FC10E947C2C809101018A3009F447
:1009500096C1843109F493C1289A60ED77E07093D1
:10096000E0036093DF0395E5909365064BEE51E05D
:100970005F934F931F920E94990EA0909C070F9037
:100980000F900F90A2FE78C189EF91E09F938F9313
:100990001F920E94990E0F900F900F90ADE0B2E061
:1009A000BF93AF931F920E94990E0E94EF1888E8A0
:1009B00093E190939D0380939C03F1E0F093640690
:1009C0000F900F900F905091E303552309F497C0B7
:1009D0001092E30320916306222309F4CDC0B09165
:1009E0009407EB2FFF27EE0FFF1FEA59F84F008106
:1009F00011810D5E1F4F14F0109202014081518150
:100A00004A5B5F4F9CF470910201772379F411E007
:100A100010930201210F20936306253008F4BCC017
:100A2000E8EEF3E0F093E003E093DF03E22EFF242F
:100A3000F0923107E09230070E940A3120910101C3
:100A40002A3009F473C0243109F470C0289A8091C7
:100A50000E03882309F45BC0815080930E0330910C
:100A60004504332329F09091450491509093450417
:100A700080919C0390919D03892B09F45BC0E091C8
:100A80009C03F0919D033197F0939D03E0939C03A9
:100A90002A3009F44DC0243109F44AC0289AD09074
:100AA000E303DD2021F0F0903C04FF2011F40E94CC
:100AB000100C0E944809CE010E9403138823E9F01C
:100AC000F091AC07AF2EBB24C0912203D091230339
:100AD000CA15DB0544F440911103509112034F5F96
:100AE0005F4F09F44CC00E94145954E05093DE0348
:100AF00084E190E00E94D212EC010E947C5AB091F5
:100B0000DE03BB2309F05FCF0E9458595CCF80936E
:100B10006F06109223041092220410922104109266
:100B2000200410921F0410921E0499CF28988FCF92
:100B30002898B5CF25E030E030939D0320939C03A7
:100B40000E941F1F60911103709112036F5F7F4F0E
:100B500009F0A5CFB0903C04BB2009F4A0CF00E180
:100B600017E21093E0030093DF03A0E8B0E0B09336
:100B70001203A093110393CF0E94B0345DCF60E7BE
:100B800077E17093E0036093DF0380E093E090935C
:100B9000120380931103A7CF822F0E94602320911C
:100BA000630644CF0E94782131E0D32E22E0E22E6A
:100BB00020E0F22E96E5A92EB12CE2E0DE1609F433
:100BC00090C033E0D31609F48FC053E05D1508F4EC
:100BD00088C02D2DE4E9F7E036E585E08D1560F558
:100BE000282F822F992701978A9DD0018B9DB00DC8
:100BF0009A9DB00D1124AC59BF4F132E0E949D60D9
:100C0000822F2630B0F085E0D701082E0E94916037
:100C10000E944A5AD394B5E0BD1578F673E0D70127
:100C2000072E0E94916069E4D801062E0E9491600F
:100C30001ECE222369F3E8CFDD2061F3D2CFD801A5
:100C40000E948460802D893409F406CE42E451E08C
:100C50005F934F931F920E94990EFBCD0E945320E9
:100C600059CE08E811E01F930F931F920E94990E2E
:100C70000F900F900F9003CE85E092E087CE2898DA
:100C80006CCEC7ECD1E0DF93CF931F920E94990EF8
:100C900088EE93E00E94D212EC010E9480140F9023
:100CA0000F900F90CE010E9403138823D9F324EEF6
:100CB00031E03F932F931F920E94990E0F900F9057
:100CC0000F9040CE87E091E02BCE29988FCD2898C9
:100CD00049CD2BE010CD199B02C024E10CCD2AE0B8
:100CE0000ACD0E941A2275CF0E94BF2272CF1F9296
:100CF0000F920FB60F9211242F938F939F93EF9320
:100D0000FF93809110038823A9F48091D4039091DC
:100D1000D5030196FC01EB5DFA4FE081ED3079F0EF
:100D20008639910561F09093D5038093D403E093C5
:100D3000C6000EC01092D5031092D40309C01092C1
:100D4000D5031092D40321E020931003E093C60052
:100D5000FF91EF919F918F912F910F900FBE0F9068
:100D60001F9018951F920F920FB60F9211242F9378
:100D70003F934F935F936F937F938F939F93AF9323
:100D8000BF93EF93FF938091C6008093CC03509163
:100D9000DA03563910F01092DB032091CC032D308A
:100DA00091F02091DB03822F99278130910509F47E
:100DB0006AC0823091050CF48CC0029709F47DC0A2
:100DC0001092DB03A6C02091DB03223061F7109262
:100DD000DB03652F77276E58794FFB013297A0818F
:100DE0002091D6033091D7032A1B3109DB011197DB
:100DF0004C91241B3109C9019F709093D7038093B4
:100E0000D6030024880F991F001C880F991F001C0F
:100E1000892F902D982F935C9093D8032F73307067
:100E2000235C2093D9033081391709F46CC090E01A
:100E3000B091C903BF5FB093C903F091CB03FF2307
:100E400009F067C0992309F464C021E02093CB0323
:100E5000520F5093C8035150E52FFF27EE58F94F1A
:100E60008DE0808350917406523509F052C048E1FC
:100E700050E09CE00FB6F894A895409360000FBE38
:100E80009093600046C02F5F2093DB03E52FFF2780
:100E9000EE58F94F8091CC0380835F5F5093DA0363
:100EA000F091CC038091D6039091D7038F0F911DC1
:100EB0009093D7038093D6032CC0E52FFF27EE58DD
:100EC000F94F2091CC032083563938F31092DB037D
:100ED000E7CF892B09F074CF3091CC03333259F02E
:100EE000B091CC03B093720671E07093DA038091F5
:100EF000CC039927DDCF6091CB03662389F7A1E06E
:100F0000A093DB03EDCF7C91721709F090CF91E0B5
:100F100094CFFF91EF91BF91AF919F918F917F916E
:100F20006F915F914F913F912F910F900FBE0F9056
:100F30001F901895BC0120E030E0A901281739075F
:100F400050F4E5E2F5E08191480F511D2F5F3F4FCE
:100F500026173707C0F3CA019F70F901EB5DFA4FFE
:100F60000024880F991F001C880F991F001C892FCF
:100F7000902D835C8083F9013196DF01AB5DBA4F20
:100F80004F735070542F535C5C93EA5DFA4F3DE011
:100F9000308310921003209125052093C6000895F8
:100FA000AF92BF92DF92EF92FF920F931F93CF9376
:100FB000DF93CDB7DEB72C859D853E8500E083E2CB
:100FC000809325059F59909326052093270563E07C
:100FD00070E0332309F498C0EF84F888B3E1AB2EB6
:100FE000B12CAC0EBD1EA989BA89D32EDA94109704
:100FF00009F48AC01097D9F1F701E00FF11D0F5FD6
:101000009081119781F4DD2099F1F5013296D50197
:10101000ED90FC90A2E0AA2EB12CAE0EBF1EA081D6
:10102000B18100E0DA94109719F1F701E00FF11D9A
:101030000F5F4081119709F478C01097D1F0F70144
:10104000E00FF11D0F5F10811197A1F4DD2091F0E9
:10105000F5013296D501ED90FC9032E0A32EB12C33
:10106000AE0EBF1EA081B18100E0DA9403C090E013
:1010700040E010E0FB01EB5DFA4F392F36953695D5
:10108000335C30836F5F7F4FFB01EB5DFA4F892F3D
:1010900099278370907082959295907F9827807F92
:1010A000982755279A01329522952F7023273F7054
:1010B0002327822B835C80839B012F5F3F4FF901A5
:1010C000EB5DFA4F4F705070440F551F440F551F82
:1010D000812F99270024880F991F001C880F991FC2
:1010E000001C892F902D842B835C8083C90101967D
:1010F000FC01EB5DFA4F1F73135C1083BC016F5F43
:101100007F4F109709F076CF20E030E0A901261735
:101110003707E8F4E5E2F5E0A1904A0D511D2F5F95
:101120003F4F26173707C0F312C0DD2009F4A1CFC7
:10113000F5013296D501ED90FC9052E0A52EB12C30
:10114000AE0EBF1EA081B18100E0DA9476CFCA0155
:101150009F70F901EB5DFA4F0024880F991F001C66
:10116000880F991F001C892F902D835C8083F901C3
:101170003196DF01AB5DBA4F4F735070142F135C83
:101180001C93EA5DFA4F0DE0008310921003B090BB
:101190002505B092C600DF91CF911F910F91FF906E
:1011A000EF90DF90BF90AF90089573E0A72F60910C
:1011B000C803665009F462C0EA2FFF27EE58F94FC2
:1011C00090819D538A2F8F5FE82FFF27EE58F94FAC
:1011D00020812D538F5FE82FFF27EE58F94F308184
:1011E0003D538F5FE82FFF27EE58F94F50815D5335
:1011F000AC5F892F9927880F991F880F991F422F5D
:1012000042954F70482B822F99278F70907082954E
:101210009295907F9827807F9827232F2695269553
:10122000282B832F9927837090700024969587959B
:101230000794969587950794982F802D582B862F85
:1012400081508F3FD9F0E72FFF27EE58F94F4083A9
:101250007F5F81508F3F91F0E72FFF27EE58F94FC6
:1012600020837F5F63506F3F49F0E72FFF27EE58E1
:10127000F94F50837F5F662309F09ECF45E756E024
:101280005093C7034093C60373507093C5030895EA
:10129000CF93DF93CDB7DEB722970FB6F894DEBFBA
:1012A0000FBECDBF8091CB03882309F462C273E0E7
:1012B000A72F6091C803665009F462C0EA2FFF2788
:1012C000EE58F94F90819D534A2F4F5FE42FFF272F
:1012D000EE58F94F20812D534F5FE42FFF27EE5832
:1012E000F94F30813D534F5FE42FFF27EE58F94F00
:1012F00050815D53AC5F892F9927880F991F880F04
:10130000991F422F42954F70482B822F99278F703B
:10131000907082959295907F9827807F9827232FB1
:1013200026952695282B832F99278370907000246B
:10133000969587950794969587950794982F802D75
:10134000582B862F81508F3FD9F0E72FFF27EE587B
:10135000F94F40837F5F81508F3F91F0E72FFF2748
:10136000EE58F94F20837F5F63506F3F49F0E72FBE
:10137000FF27EE58F94F50837F5F662309F09ECF19
:10138000A5E7B6E0B093C703A093C603735070936C
:10139000C50350917306523609F460C080917406FB
:1013A00099278736910579F188369105C4F58136FC
:1013B000910509F492C0823691050CF072C08B340D
:1013C000910521F5E091C603F091C703A081B18199
:1013D000B0935804A09357048091570490915804F7
:1013E0004091550450915604841B950B845E9D4F8B
:1013F00068E671E00E943460845B904090935404EE
:101400008093530403C081E08093D3031092CB03F5
:101410001092C7031092C6031092C503AAC18C365E
:10142000910509F467C08D3691057CF588369105E4
:1014300069F73FEF30930E03E091C603F091C703C5
:101440007081F0910B047F2B70930B04772311F0C4
:101450001092CD0351E05093D103D8CF8091740600
:1014600099278137910509F431C1823791050CF034
:101470004FC08B34910509F49EC08037910509F067
:101480008DCF91E09093CE0389CF8437910509F4F5
:101490006FC08637910509F0B9CFA1E0A093CF03C3
:1014A000B5CF8236910509F453C08436910509F011
:1014B000ADCFE091C603F091C70390818AE0989F79
:1014C000F0011124F0930C03E0930B03EF2B09F4CC
:1014D0009DCF21E02093D00399CFE091C603F091F6
:1014E000C703E081E03280F5E0930F036FEF609374
:1014F0000E038CCFBFEFB0930E03E091C603F091C3
:10150000C703908190930C0441E04093D2037ECFB7
:101510008337910509F46EC08437910509F03ECFF9
:101520008091750690917606A0917706B091780625
:101530008093C0039093C103A093C203B093C303ED
:101540007FEF70930E032ACF9FE190930F03CECFCE
:10155000A091C603B091C7038BE0E5E6F6E00D90DD
:1015600001928A95E1F7B0916E06B0934A07BECF1B
:10157000E091C603F091C7032081318142815381FC
:101580002093C0033093C1034093C2035093C3031D
:10159000709110037723E1F31F9250910D035F9335
:1015A00034E53F930E94D007FFEFF0930E030F90B6
:1015B0000F900F902BCFA0917506B0917606B09347
:1015C0005804A09357048091570490915804609157
:1015D000550470915604861B970B845E9D4F68E6F8
:1015E00071E00E943460845B904090935404809337
:1015F0005304D4CE90917506F92FF150F53020F4B4
:10160000309176063934E9F01A82909110039923CB
:10161000E1F361E070E07F936F93CE0102969F93B8
:101620008F93A1E0AF93AF93B3E5BF930E94D00730
:101630008DB79EB707960FB6F8949EBF0FBE8DBFAD
:10164000ADCE64E977E056E51296FB01452F0D908B
:1016500001924A95E1F7452F892F0E94F20280916D
:10166000BF079927AA27BB27BC01CD0124EC39E08D
:1016700040E050E00E94F55FDC01CB0180939603CF
:1016800090939703A0939803B09399038091C00718
:101690009927AA27BB27BC01CD010E94F55FDC0179
:1016A000CB018093920390939303A0939403B09300
:1016B0009503E091C603F091C70380810E94E60282
:1016C0000E9420038A830E9460239FCFB0917506F9
:1016D000BF3F09F446C0E091C603F091C703808183
:1016E0008823D9F581E08083E091C603F091C70398
:1016F00046E564E977E080810E94C902F091100319
:10170000FF23E1F3E091C603F091C70370817A8370
:1017100059E4598326E530E03F932F93E4E9F7E05D
:10172000FF93EF9361E070E07F936F93CE01860F9C
:10173000971F9F938F937F936F93DE011296BF93B2
:10174000AF9343E04F9321E02F9331E53F930E9405
:10175000D0078DB79EB70F966ECF863048F285E0E2
:10176000C2CF0E942003E091C603F091C70380839B
:10177000B2CF22960FB6F894DEBF0FBECDBFDF9179
:10178000CF910895CF93C82F8A3029F08091C0005F
:1017900085FFFCCF04C08DE00E94C20BF7CFC09341
:1017A000C60080E090E0CF910895089578E17093AD
:1017B000C1006091C00062606093C0005091C100A0
:1017C00050685093C1004091C10040644093C100F3
:1017D0003AE23093C40080910B0390910C030E9475
:1017E000D21290935206809351068CED90E00E94A5
:1017F000D21290937106809370061092530627E4DC
:10180000209354068AE080935706809355061092E1
:1018100056061092C7031092C6031092C50308958E
:1018200080911003882309F47EC02091D1032223E4
:1018300009F07AC09091D203992329F0B091100356
:10184000BB2309F06DC15091CF03552329F070914E
:101850001003772309F049C1F091D303FF2329F046
:1018600030911003332309F024C1809170069091C8
:1018700071060E940313882329F0709110037723C7
:1018800009F0BFC0E0910B03F0910C03EF2B09F0BE
:1018900072C16091D003662329F070911003772301
:1018A00009F073C120910F032F3F61F140E150E037
:1018B0005F934F93A22FBB27A295B295B07FBA2713
:1018C000A07FBA27A55FBE4FBF93AF9381E090E0A2
:1018D0009F938F936FE073E07F936F93E2E0EF93BA
:1018E00051E05F9331E43F930E94D007FFEFF09304
:1018F0000F034DB75EB7455F5F4F0FB6F8945EBFFD
:101900000FBE4DBF70914A07772329F090911003C5
:10191000992309F05CC0F091CE03FF2321F03091B0
:1019200010033323D1F5089530911003332309F4C4
:1019300081CF0E94F81824E130E03F932F939091DB
:10194000CD0384E1989FC00111248B5D9C4F9F9330
:101950008F93E1E0F0E0FF93EF93ADECB3E0BF9342
:10196000AF9372E07F9361E06F9358E45F930E94BE
:10197000D0078091CD038F5F4DB75EB7455F5F4F56
:101980000FB6F8945EBF0FBE4DBF843008F424C17B
:101990001092CD031092D1034DCF26E130E03F935A
:1019A0002F93E6E6F7E0FF93EF9341E04F934F93D9
:1019B00050E55F930E94D0071092CE03ADB7BEB73B
:1019C00017960FB6F894BEBF0FBEADBF089581E065
:1019D00090E09F938F936AE477E07F936F9321E089
:1019E0002F932F93B2E4BF930E94D00710924A071F
:1019F000EDB7FEB737960FB6F894FEBF0FBEEDBF3A
:101A00008ACF8091910490919204A0919304B09117
:101A10009404BC01CD012CE630E040E050E00E948F
:101A2000696030935E0620935D06809189049091F1
:101A30008A04A0918B04B0918C04BC01CD012CE6EA
:101A400030E040E050E00E946960309360062093EF
:101A50005F0650912D0450936106A0912C04A09331
:101A6000620628E030E03F932F938DE596E09F9348
:101A70008F9331E03F93F3E0FF93B7E7BF930E946A
:101A8000D00790916306EDB7FEB737960FB6F8947E
:101A9000FEBF0FBEEDBF953018F046E040936306E1
:101AA00083E690E00E94D2129093710680937006B4
:101AB000E9CE6BE070E07F936F9345E656E05F936D
:101AC0004F9351E05F93A0910D03AF9327E42F93C1
:101AD0000E94D0071092D3038DB79EB707960FB61A
:101AE000F8949EBF0FBE8DBFC0CEEAE0F0E0FF933A
:101AF000EF9363E576E07F936F93B1E0BF93BF937D
:101B000096E59F930E94D0071092CF034DB75EB722
:101B1000495F5F4F0FB6F8945EBF0FBE4DBF9CCEBE
:101B20000E94F818A0E5B0E0BF93AF9325E233E040
:101B30003F932F93E1E0F0E0FF93EF9384E293E093
:101B40009F938F93FF93EF936CE074E07F936F9379
:101B500043E04F9331E03F93FCE4FF930E94D007B2
:101B60001092D203ADB7BEB71F960FB6F894BEBFA2
:101B70000FBEADBF68CE80915106909152060E9473
:101B80000313882309F089CE84CEA2E4B0E0BF938A
:101B9000AF9328E037E03F932F93B1E0BF93BF931B
:101BA00094E49F930E94D0071092D0038DB79EB704
:101BB00007960FB6F8949EBF0FBE8DBF80910B03A2
:101BC00090910C03009709F46DCE0E94D21290936D
:101BD00052068093510666CE8093CD031092D103B6
:101BE00029CE982F80914B07813031F0892F0E94A8
:101BF000C20B282F33270CC020910D04E22FFF27A2
:101C0000EB5DFC4F90832F5F20930D0421E030E0CB
:101C1000C90108950F931F93CF93DF938C01EB01BC
:101C2000672B69F418C020910D04E22FFF27EB5DAC
:101C3000FC4F90832F5F20930D04219761F0F801F2
:101C400091918F0180914B07813069F3892F0E9418
:101C5000C20B2197A1F7DF91CF911F910F910895AA
:101C60000F931F93CF93DF938C01EB01672B69F4E4
:101C700019C020910D04E22FFF27EB5DFC4F9083EC
:101C80002F5F20930D04219769F0F8010F5F1F4F1C
:101C9000949180914B07813061F3892F0E94C20B90
:101CA000219799F7DF91CF911F910F9108951F937D
:101CB000CF93C82F1816CCF410E20DC020910D045C
:101CC000E22FFF27EB5DFC4F10832F5F20930D0465
:101CD000C1501C1654F480914B07813079F380E297
:101CE0000E94C20BC1501C16B4F3CF911F910895EE
:101CF0001F93CF93C82F1816CCF410E30DC020917A
:101D00000D04E22FFF27EB5DFC4F10832F5F209324
:101D10000D04C1501C1654F480914B07813079F3A7
:101D200080E30E94C20BC1501C16B4F3CF911F91E7
:101D300008952F923F924F925F926F927F928F926F
:101D40009F92AF92BF92CF92DF92EF92FF920F934A
:101D50001F93CF93DF93CDB7DEB7E3970FB6F89419
:101D6000DEBF0FBECDBF29968FAD29972B96EEAD66
:101D7000FFAD2B9788249924540180934B077BE473
:101D8000C72ED12CCC0EDD1E7F019701F701549098
:101D9000552039F0F5E25F1621F00894E11CF11CA2
:101DA000F5CFC701821B930BE9F039018C010DC0FF
:101DB00030910D04E32FFF27EB5DFC4F90833F5FD5
:101DC00030930D040150104069F0F3010894611C38
:101DD000711C949120914B07213051F3892F0E945F
:101DE000C20BF0CF552009F4DAC20894E11CF11CB3
:101DF0001FA60FA5202E6FEF762E09A7F7010894D6
:101E0000E11CF11C14911537C9F1412F406248378C
:101E1000A9F1103209F440C0133209F488C01A3213
:101E200009F476C01D3209F473C01B32C9F11E32A9
:101E3000C9F1103309F483C0712F7153793008F060
:101E400078C020E030E01901220C331C220C331C36
:101E5000220C331C220E331E220D331D210F311D87
:101E600020533040F7010894E11CF11C1491912F8C
:101E700090539A3040F3222E153739F600FF3DC0BB
:101E8000F60164E070E0C60ED71E80809180A280CB
:101E9000B380103209F0C0CF39A4332009F0AECF9F
:101EA00019A7ACCFF7010894E11CF11C14911A3268
:101EB00009F449C020E030E014C03901660C771CF9
:101EC000660C771C660C771C620E731E260D371D80
:101ED000210F311D20533040F7010894E11CF11C03
:101EE0001491512F50535A3040F3C9012F5F3F4F87
:101EF00014F48FEF9FEF782E86CFF601A2E0B0E0CA
:101F0000CA0EDB1E408051804201AA24BB2481CF2F
:101F10001A3251F4F60182E090E0C80ED91E2080FA
:101F200022200CF06BCF219400610F7D67CF0860F9
:101F300065CF1836B9F01C36B9F401605FCF04FDE7
:101F40005DCF00625BCFF60122E030E0C20ED31E0F
:101F500080819181EFEF8F3F9E0714F48FEF9FEF09
:101F6000782E4CCF04604ACF133609F40CC21434D7
:101F700009F4DFC1143609F4DCC1193609F4D9C1FA
:101F80001F3409F4D0C11F3609F4CDC1103709F44C
:101F9000BBC1133709F47CC1153509F473C115377A
:101FA00009F470C1183509F407C1183709F404C1E0
:101FB000112309F4F4C1DE011196BDA7ACA7198362
:101FC00091E0392E19A6602E7724832D5FA4531833
:101FD00057FCF0C029A5222309F4C5C0832D8F5FCB
:101FE000850D8BABC30180739070892BF1F4022DAA
:101FF000BBA90B1B1016CCF480E2482E0DC030910B
:102000000D04E32FFF27EB5DFC4F40823F5F3093D1
:102010000D040150101644F4F0914B07F13079F3A0
:1020200080E20E94C20BF5CF29A5222309F474C0D7
:1020300099A510914B07113009F0B8C020910D04FB
:10204000E22FFF27EB5DFC4F90832F5F20930D0461
:102050008301007310700032110509F489C0152D39
:102060001514BCF400E30DC0B0910D04EB2FFF2755
:10207000EB5DFC4F0083BF5FB0930D041150111650
:1020800044F480914B07813079F380E30E94C20BC6
:10209000F5CF4CA45DA4032D112707FD1095011564
:1020A0001105D1F0F20191912F01F0914B07F13020
:1020B00069F430910D04E32FFF27EB5DFC4F908313
:1020C0003F5F30930D0401501040E9CF892F0E94EB
:1020D000C20B01501040E3CF64FE57CE122D2BA847
:1020E000121911160CF051CE00E20EC0A0910D0491
:1020F000EA2FFF27EB5DFC4F0083AF5FA0930D0439
:10210000115011160CF041CE20914B07213071F384
:1021100080E20E94C20BF4CF66FE9ACF40E34AA74A
:102120001BA7DE019A96BAABA9AB02E010E00EC085
:1021300050910D04E52FFF27EB5DFC4F90835F5F0F
:1021400050930D040150104009F482CFE9A9FAA977
:102150009191FAABE9AB60914B07613049F3892F5C
:102160000E94C20BEFCF66FE3BCF832D8E5F38CF30
:10217000122D4BA8141911160CF071CF00E30EC0EC
:1021800090910D04E92FFF27EB5DFC4F00839F5FCB
:1021900090930D04115011160CF061CF70914B0704
:1021A000713071F380E30E94C20BF4CF892F0E943B
:1021B000C20B4ECF55240ECF30E13EA703FF06C021
:1021C00081149104A104B10409F0006419A67FA64A
:1021D00077FE0F7DDE019996BDA7ACA7811491040F
:1021E000A104B10419F45FA4552069F12EA5422E73
:1021F00055246624772418AA84149504A604B704E9
:1022000010F041E048ABC501B401A30192010E9466
:102210004760DC01CB018A3000F530E3332E380E05
:10222000ECA5FDA53292FDA7ECA7C501B401A30161
:1022300092010E94476049015A0158A95523D9F6D5
:102240007EA5783091F0602E7724CE010196382E4D
:102250009CA5391A08E2300EB8CE27E5322E380E8A
:102260001835F1F66FED3622DBCF602E772463FE52
:10227000ECCF80E3381649F3ECA5FDA58293FDA7CA
:10228000ECA7E3CF153509F40160FAE0FEA79ECF75
:10229000F60162E070E0C60ED71EA081B181BDA735
:1022A000ACA7AB2B81F4FE013196FDA7ECA7B8E2F9
:1022B000B9838EE6818395E79B837CE67C837D836F
:1022C00059E25E831F8277FC15C0472C552447FCDA
:1022D0005094A20160E070E08CA59DA50E94805EF4
:1022E000009731F0382E6CA4361873140CF06ACEB7
:1022F000372C68CEECA5FDA501900020E9F73197B9
:102300003E2E7CA437185ECEF60142E050E0C40EAB
:10231000D51E208131814901AA24BB2410E11EA7CA
:10232000006418E753CF1F3409F4016038E03EA77A
:102330004DCF143409F4016000FF18C0F60164E0C9
:1023400070E0C60ED71E80809180A280B380B7FE59
:102350000AC0B094A09490948094811C911CA11CFC
:10236000B11CBDE2B9A7FAE0FEA731CFF60182E0C9
:1023700090E0C80ED91E408051804201AA2497FCEB
:10238000A094BA2CE4CFDE011196BDA7ACA7F6014C
:1023900042E050E0C40ED51E5080598211CEE39623
:1023A0000FB6F894DEBF0FBECDBFDF91CF911F9166
:1023B0000F91FF90EF90DF90CF90BF90AF909F90E4
:1023C0008F907F906F905F904F903F902F900895E7
:1023D0001F920F920FB60F9211242F933F934F939A
:1023E0005F936F937F938F939F93AF93BF93EF937D
:1023F000FF938091DE03882329F02091DE03215092
:102400002093DE038091E60381508F3F09F495C04D
:102410008093E6036091DF037091E0036230710501
:1024200000F1A091DF03B091E0031197B093E003B6
:10243000A093DF03E091DF03F091E00380911103AB
:1024400090911203E823F923EF2B89F07091010199
:102450007A3009F48FC0479AB0919C07B3FF91C0BE
:1024600010C02FEF3FEF3093120320931103909190
:1024700001019A3009F47AC04798B0919C07B3FFE4
:1024800080C086B19927FC01E071F07084FF0AC01A
:10249000E091E103F091E2033196F093E203E093DF
:1024A000E1036FC08091E1039091E203892B51F128
:1024B0004091E1035091E2034A56514018F5809152
:1024C000E1039091E20369E270E00E942060A09134
:1024D000E103B091E203A60FB71FB093E203A0930C
:1024E000E1036091E1037091E2036B30710508F440
:1024F00043C0E091E103F091E2033A97F09358046E
:10250000E0935704809157049091580440915504EA
:1025100050915604841B950B845E9D4F68E671E0D4
:102520000E943460845B90409093540480935304E1
:102530001092E2031092E10324C049E04093E603C5
:1025400090E030911503332399F09093150399236C
:1025500019F451E05093E303A091E403B091E50333
:102560001196B093E503A093E40354CF5A9885CF16
:1025700091E0EBCF5A9A81CFF0935804E09357043F
:10258000C1CFFF91EF91BF91AF919F918F917F91BB
:102590006F915F914F913F912F910F900FBE0F90D0
:1025A0001F9018952091E4033091E503280F391FFF
:1025B000C90101960895E091E403F091E5033B968B
:1025C000F093E803E093E703A2E0A5BD93EA94BD8E
:1025D00017BC78E778BD66E066BD53EC5093B00059
:1025E00044E04093B100309170003260309370004D
:1025F00020916E00216020936E008AE08093B300EA
:102600001092B20008952091E4033091E503821BFB
:10261000930B892F99278695807490700895209147
:10262000E4033091E503280F391F2F5F3F4F60917E
:10263000E4037091E503A901461B570B57FFF7CF41
:1026400008952091E4033091E503280F391F2F5F8F
:102650003F4F6091E4037091E503A901461B570BBE
:1026600057FD0CC04FEE40937A008091E4039091A7
:10267000E503F901E81BF90BF7FFF5CF08951F9269
:102680000F920FB60F9211242F933F938F939F9326
:102690008091130390911403892B11F05F9A01C06C
:1026A0005F9833E03093B000209170002E7F20932C
:1026B00070009F918F913F912F910F900FBE0F90BF
:1026C0001F9018951F920F920FB60F9211242F93FF
:1026D0003F934F935F936F937F938F939F93AF93AA
:1026E000BF93CF93DF93EF93FF9380911303909168
:1026F00014030497C1F1C0911303D0911403CD2B9F
:10270000B9F48091130390911403892B09F0D6C07A
:102710008091B9079927880F991F880F991F909367
:102720001403809313035F9883E08093B000C6C0C6
:1027300060911303709114036430710510F72091B8
:10274000DC033091DD032F3F310509F008F49BC015
:102750005F9A53E05093B0002F5F30403093DD0319
:102760002093DC03ABC040911703509118039A01EA
:10277000220F331F240F351F809184039927880F60
:10278000991F280F391F37FD8CC0D901B595A79522
:10279000B595A795B0931803A0931703ED01E096A4
:1027A0008091B70723E0829FC0011124C817D90781
:1027B000E0F5EC012091DA0720FF47C08091B607D1
:1027C0009927AA27BB272091910430919204409128
:1027D000930450919404BC01CD010E94F55F97FDD4
:1027E00063C05EE095958795779567955A95D1F783
:1027F0009E01260F371F3093330720933207C901FC
:102800006FEF70E00E9420608D97C8F4235B3F4F0C
:102810003093DD032093DC0383E180931603322F92
:1028200030953093B30083EC80CF8091B807829FBE
:10283000C00111248C179D0708F0BCCFBACF30938C
:10284000DD032093DC0380E6E8CF8091B60799276B
:10285000AA27BB27209191043091920440919304C0
:1028600050919404BC01CD010E94F55F97FD21C0F9
:102870004EE095958795779567954A95D1F79E0196
:10288000261B370BB8CF93E89093B00070911603D6
:102890007093B300E1E0F0E0F0931403E0931303CE
:1028A0000DC02D5F3F4F71CF6150704C8F4F9F4FC8
:1028B00098CF6150704C8F4F9F4FDACFA091130388
:1028C000B09114031197B0931403A0931303FF91D5
:1028D000EF91DF91CF91BF91AF919F918F917F91B8
:1028E0006F915F914F913F912F910F900FBE0F907D
:1028F0001F90189510927C008FEE80937A000895B7
:10290000EF92FF920F931F93CF93DF9303E010E0BA
:10291000D8010E948460802DC82FDD27C531D105E4
:1029200008F02A97C7BD1092F00384E690E00E9459
:10293000211340911C0350911D034255534010F444
:10294000C0E0D0E0CA3FD105E0F481E1E82E82E0AA
:10295000F82EC7BD82E390E00E942113FF92EF9210
:102960001F920E94990E60911C0370911D030F909D
:102970000F900F906255734020F02196CA3FD10509
:1029800040F3D8010C2E0E949160C09359078CE24D
:1029900091E00E942113DF91CF911F910F91FF9041
:1029A000EF900895FF920F931F93CF9310E0109331
:1029B000EB031093EA031093E903CCE801E095EFF1
:1029C000F92E133009F499C010E080910104909120
:1029D00002048C5F93400CF07FC080911B038150F8
:1029E00080931B036091FF03709100046C5F734040
:1029F0000CF067C080911A03815080931A03E09114
:102A0000FD03F091FE03EC5FF340D4F580911903D0
:102A100081508093190328E0209312040E940B1F19
:102A200080911B038A3008F044C00093EB033AE026
:102A300030931B0380911A038A30A0F50093EA03B8
:102A40005AE050931A03809119038A3020F50093BD
:102A5000E9037AE070931903809112048823E1F767
:102A6000809354079FEE90937A00B0915407BB2354
:102A7000E1F3CA3008F446C0C15009F0A2CF47C004
:102A80008091FD039091FE038750944084F18091E2
:102A900019038F5FBECF863FF8F20093E903F092EF
:102AA0001903DACF863F78F20093EA03F0921A0313
:102AB000CACF863F08F4BECF0093EB03F0921B030E
:102AC000B9CFA091FF03B0910004A750B4408CF09F
:102AD00080911A038F5F91CF4091010450910204BD
:102AE0004750544044F080911B038F5F79CF1F5FA4
:102AF00092CF1F5F84CF11E075CFCB3008F464CF45
:102B0000C9E062CF8AE090E00E942113B5CF86E44D
:102B100090E00E942113CF911F910F91FF90089593
:102B20001F920F920FB60F921124EF92FF920F9304
:102B30001F932F933F934F935F936F937F938F9345
:102B40009F93AF93BF93CF93DF93EF93FF93109235
:102B50007A0080910404682F77278F5F65307105B4
:102B600009F440C066307105ACF46230710509F4B7
:102B700048C1633071050CF45CC06330710509F421
:102B800049C26430710509F471C2109203041092B5
:102B9000040442C06830710509F41AC16930710536
:102BA0000CF05BC06630710509F450C167307105E7
:102BB00061F780930404109101011A3009F4D0C226
:102BC0008091780090917900409107045091080419
:102BD000840F951F909300048093FF0382E08093FD
:102BE00003041AC080930404409178005091790046
:102BF00020919F043091A004421B530B509358071F
:102C000040935707E0905707F0905807F092FA0367
:102C1000E092F903109203041091030410937C00D6
:102C2000F0900404FF2009F4C3C23FEE30937A0011
:102C3000BFC26115710509F4F2C06130710509F078
:102C4000A4CF8093040420917800309179003093D0
:102C500008042093070482E0C2CF6930710509F4AB
:102C600011C16A30710509F090CFA0917800B09140
:102C7000790000915C0710915D07A00FB11FB09320
:102C80005D07A0935C07909154079F5F9093540752
:102C900070915407753008F478CF60917800709186
:102CA000790070931D0360931C03109254070091E8
:102CB000EE031091EF03B801660F771F660F771FC1
:102CC000660F771F601B710BF0918D03EF2EFF24B1
:102CD000B091F003EB2FFF27E7FDF095AFEFB0E0E9
:102CE000EA9F8001EB9F100DFA9F100D1124809137
:102CF000500790915107800F911FC0915C07D091B0
:102D00005D078C1B9D0B40913A0450913B04841B42
:102D1000950BE89E9001E99E300DF89E300D112430
:102D2000620F731F77FD41C275956795759567951D
:102D3000759567957093EF036093EE03E0905C07E1
:102D4000F0905D07E701EE27D7FDE095FE2F20917B
:102D50001E0330911F034091200350912103DA019B
:102D6000C901880F991FAA1FBB1F820F931FA41FA1
:102D7000B51FC80FD91FEA1FFB1FF7FD12C2F5953B
:102D8000E795D795C795F595E795D795C795C093DE
:102D90001E03D0931F03E0932003F0932103C091FF
:102DA0005007D0915107C00FD11F20911E033091C1
:102DB0001F034091200350912103C21BD30BD093DA
:102DC0003B04C0933A0410925D0710925C07DDCE7D
:102DD00080930404309101013A3009F43AC18091A2
:102DE000780090917900C0910904D0910A048C0F69
:102DF0009D1F909302048093010485E08093030457
:102E00000BCF809304044091780050917900509347
:102E10000A044093090484E080930304FDCE809368
:102E20000404E0907800F0907900F0920604E092BB
:102E3000050401E0009303048091EC039091ED03FD
:102E400001969093ED038093EC03E6CE8093040407
:102E5000809101018A3009F471C1843109F48DC176
:102E600080917800909179000091050410910604FA
:102E7000800F911F9093FE038093FD0381E0809368
:102E80000304CACE80930404809178009091790065
:102E9000AA2797FDA095BA2FBC01CD010E94335FF0
:102EA000C0919704D0919804E0919904F0919A040C
:102EB0009E01AF010E948D5EDC01CB01BC01CD0102
:102EC0000E94165FDC01CB019093F8038093F70317
:102ED0008091F7039091F80302970CF4E3C080917E
:102EE000970490919804A0919904B0919A0420E0DD
:102EF00030E84BE354E4BC01CD010E943D5F8823E0
:102F0000CCF58091970490919804A0919904B09188
:102F10009A042AE037ED43EA5CE3BC01CD010E944C
:102F20008E5E6093970470939804809399049093B5
:102F30009A04A0911804B0911904A45FB140D0F490
:102F40008091970490919804A0919904B0919A046B
:102F50002DEC3CEC4CEC5DE3BC01CD010E948E5E9F
:102F6000DC01CB018093970490939804A09399047B
:102F7000B0939A0451E05093F1034091780050913E
:102F8000790050934F0740934E078091F70390913B
:102F9000F803AA2797FDA095BA2FE0905904F09066
:102FA0005A0400915B0410915C048E0D9F1DA01FBC
:102FB000B11F8093590490935A04A0935B04B0937B
:102FC0005C042091590430915A0440915B04509163
:102FD0005C0457FDC0C0AAE05595479537952795E5
:102FE000AA95D1F7C0915904D0915A04E0915B049D
:102FF000F0915C04C21BD30BE40BF50BC093590496
:10300000D0935A04E0935B04F0935C0483E08093D4
:10301000030402CE80930404E0912203F091230381
:10302000EF01CC0FDD1FCE0FDF1F80917800909154
:1030300079000E942060C60FD71FD695C795D695F8
:10304000C795D0932303C093220386E080930304A3
:10305000E3CD80917800909179002091090430911E
:103060000A04820F931F96958795C3CE809304041C
:1030700080919D0490919E040091780010917900B8
:10308000801B910B90934D0780934C0760914C07E8
:1030900070914D077093FC036093FB0387E080936E
:1030A0000304BACDE091F703F091F803EF5FFF4F0F
:1030B0000CF060CF8091970490919804A0919904AE
:1030C000B0919A0420E030E849E054E4BC01CD011D
:1030D0000E94405F18160CF04DCF8091970490919C
:1030E0009804A0919904B0919A042AE037ED43EA3C
:1030F0005CE3BC01CD010E948D5E609397047093E8
:1031000098048093990490939A04609118047091A4
:103110001904645F714008F02DCF8091970490915D
:103120009804A0919904B0919A042DEC3CEC4CECDD
:103130005DE3BC01CD010E948D5E12CF80917800CD
:1031400090917900C0910504D09106048C0F9D1FC9
:10315000969587958FCE21503C4F4F4F5F4F3BCF79
:103160008091780090917900E0900704F090080435
:103170008E0D9F1D969587952DCDE0917800F0914D
:1031800079006091050470910604E60FF71FAFEF18
:10319000B3E0AE1BBF0BB093FE03A093FD0381E031
:1031A0006ECE2396E11DF11DEACD695F7F4FBCCD48
:1031B000FF91EF91DF91CF91BF91AF919F918F914F
:1031C0007F916F915F914F913F912F911F910F913F
:1031D000FF90EF900F900FBE0F901F90189590E208
:1031E000E5E2F3E08FE49193815087FFFCCF0895EF
:1031F0001F93CF93DF9380910C0420912403281711
:1032000010F420930C0490910B0490FF08C080915F
:103210000C04882309F49FC0815080930C0491FF13
:1032200008C080910C04821709F490C18F5F8093CD
:103230000C04892F992780FF02C081FD89C090E28C
:10324000E5E2F3E08FE49193815087FFFCCF90910A
:103250000C049A3008F082C011E110930D04292F5C
:1032600033273F932F9383E192E09F938F9351E015
:103270005F930E94990E0F900F900F900F900F90F8
:1032800080910C04C82FDD27C530D10509F461C138
:10329000C630D1050CF06CC0C230D10509F4EEC1C6
:1032A000C330D1050CF0A3C0209709F49EC221972A
:1032B00009F070C0B0919C07B0FF81C510920D0459
:1032C00040913A0450913B045F934F932FE532E0D5
:1032D0003F932F9311E01F930E94990E54E1509356
:1032E0000D040F900F900F900F900F908091380465
:1032F000909139049F938F93EEE6F2E0FF93EF9362
:103300001F930E94990E38E230930D040F900F9096
:103310000F900F900F90C0911C03D0911D03DF936D
:10332000CF93ADE7B2E0BF93AF931F930E94990E86
:10333000FCE3F0930D040F900F900F900F900F90FF
:103340008091590799279F938F938CE892E049C207
:1033500010920C0474CF20930C0461CF30E13093B1
:103360000D04492F55275F934F9388E192E07DCF5D
:10337000C830D10509F4F3C1C930D1058CF0CA3089
:10338000D10509F40FC4CA30D1050CF489C22B97BA
:1033900009F4B3C481508093240310920C042FC508
:1033A000C630D10509F499C32797A1F714E110930A
:1033B0000D0460912203709123037F936F9345E482
:1033C00054E05F934F9311E01F930E94990E38E2EF
:1033D00030930D040F900F900F900F900F908091ED
:1033E000450499279F938F9384E594E0FAC1C330F5
:1033F000D10509F406C3249769F610920D043091A3
:103400009507C32FDD27CC0FDD1FCA59D84F288160
:1034100039813F932F9310919407E12FFF27EE0FEF
:10342000FF1FEA59F84FA081B181BF93AF9367E2C4
:1034300073E07F936F9311E01F930E94990EF4E164
:10344000F0930D048DB79EB707960FB6F8949EBF04
:103450000FBE8DBFB0919707CB2FDD27CC0FDD1F9F
:10346000CA59D84F488159815F934F9390919607DD
:10347000E92FFF27EE0FFF1FEA59F84F2081318116
:103480003F932F93A7E3B3E0BF93AF931F930E94A3
:10349000990E78E270930D048DB79EB707960FB61C
:1034A000F8949EBF0FBE8DBF50919907C52FDD27A1
:1034B000CC0FDD1FCA59D84F688179817F936F93F4
:1034C00030919807E32FFF27EE0FFF1FEA59F84FBF
:1034D000408151815F934F9327E433E03F932F93D3
:1034E0001F930E94990EFCE3F0930D04ADB7BEB795
:1034F00017960FB6F894BEBF0FBEADBFB0919B0735
:10350000CB2FDD27CC0FDD1FCA59D84F8881998179
:103510009F938F9390919A07E92FFF27EE0FFF1F3C
:10352000EA59F84F608171817F936F9387E593E04B
:103530009F938F931F930E94990E8DB79EB7079606
:103540000FB6F8949EBF0FBE8DBF59C410920C04E5
:1035500070CE10920D0447E653E05F934F93C1E0A5
:10356000CF930E94990E809101010F900F900F90C0
:103570008A3009F45DC38B3009F4DDC1843109F46C
:10358000DAC18D3009F03BC434E130930D048091F1
:103590001B0399279F938F932091A9043091AA042C
:1035A000C90137FD2AC4959587959F938F93809184
:1035B000010490910204821B930B9F938F932FEC35
:1035C00033E03F932F93CF930E94990E58E250938C
:1035D0000D04EDB7FEB739960FB6F894FEBF0FBED7
:1035E000EDBF80911A0399279F938F932091A70491
:1035F0003091A804C90137FDFEC3959587959F9327
:103600008F936091FF0370910004621B730B7F9393
:103610006F9343EE53E05F934F93CF930E94990EC5
:103620007CE370930D04ADB7BEB719960FB6F8944E
:10363000BEBF0FBEADBF8091190399279F938F9393
:103640002091A5043091A604C90137FDD2C39595F8
:1036500087959F938F938091FD039091FE03281B84
:10366000390B3F932F93E7EFF3E0FF93EF93CF9363
:103670000E94990E8DB79EB7099662CF10920D04E5
:10368000A0EBB2E0BF93AF93C1E0CF930E94990E3D
:1036900094E190930D040F900F900F9080919104FE
:1036A00090919204A0919304B0919404B7FD20C32B
:1036B0002AE0B595A795979587952A95D1F7BF9359
:1036C000AF939F938F938AEB92E09F938F93CF93C7
:1036D0000E94990EB8E2B0930D04EDB7FEB737968D
:1036E0000FB6F894FEBF0FBEEDBF80918904909194
:1036F0008A04A0918B04B0918C04B7FD5BC31AE0DF
:10370000B595A795979587951A95D1F7BF93AF93E0
:103710009F938F9369EC72E07F936F93CF930E9496
:10372000990EFCE3F0930D04ADB7BEB717960FB634
:10373000F894BEBF0FBEADBF4091570450915804DE
:103740005F934F9328ED32E03F932F93CF930E94E6
:10375000990E0F900F900F900F900F9050C31092F2
:103760000D0443E654E05F934F9311E01F930E94D2
:10377000990E94E190930D040F900F900F9020916B
:103780005304309154043F932F93A2E7B4E0BF93C6
:10379000AF931F930E94990E78E270930D040F90DF
:1037A0000F900F900F900F90C0915704D091580434
:1037B000DF93CF9381E894E09F938F931F930E94B0
:1037C000990E5CE350930D040F900F900F900F90A3
:1037D0000F90E0915504F0915604FF93EF9380E928
:1037E00094E09F938F931F93B2CF10920D046DE1DD
:1037F00072E07F936F9311E01F930E94990E94E102
:1038000090930D040F900F900F904BE650E05F9354
:103810004F9327E430E03F932F93DF93CF93809132
:1038200001016AE00E941460892F99279F938F936A
:10383000809101010E94146099279F938F93EDE27C
:10384000F2E0FF93EF931F930E94990E78E270933A
:103850000D04CDB7DEB72D960FB6F894DEBF0FBEC0
:10386000CDBF0E94200399279F938F93A2E4B2E0DB
:10387000BF93AF931F930E94990E6CE360930D0466
:103880000F900F900F900F900F908FE492E09F9306
:103890008F931F930E94990E0F900F900F90AFC2BD
:1038A00010920D0440914C0450914D045F934F933E
:1038B0002FE934E03F932F9311E01F930E94990E5C
:1038C00034E130930D040F900F900F900F900F90F4
:1038D000A0914A04B0914B04BF93AF93CBEAD4E0DC
:1038E000DF93CF931F930E94990EF8E2F0930D049B
:1038F0000F900F900F900F900F908091480490912F
:1039000049049F938F93E7EBF4E0FF93EF931F93AA
:103910000E94990EBCE3B0930D040F900F900F908E
:103920000F900F9060914604709147047F936F93BE
:1039300083EC94E056CFB4E1B0930D042091A90438
:103940003091AA04C90137FD52C2959587959F937E
:103950008F93E0910104F0910204E21BF30BFF93BB
:10396000EF9362EA73E07F936F93CF930E94990E77
:10397000F8E2F0930D04ADB7BEB717960FB6F89402
:10398000BEBF0FBEADBF2091A7043091A804C901EE
:1039900037FD2BC2959587959F938F93A091FF0339
:1039A000B0910004A21BB30BBF93AF9341EB53E064
:1039B0005F934F93CF930E94990E1CE310930D04D5
:1039C0008DB79EB707960FB6F8949EBF0FBE8DBFFA
:1039D0002091A5043091A604C90137FD04C2959534
:1039E00087959F938F936091FD037091FE03261B33
:1039F000370B3F932F9380EC93E09F938F93CF935C
:103A00009ACD10920D04C0916A07D0916B07DF9395
:103A1000CF9340916807509169075F934F9327EECA
:103A200032E03F932F9311E01F930E94990E74E1AF
:103A300070930D04ADB7BEB717960FB6F894BEBF1E
:103A40000FBEADBF80916E0790916F079F938F93CC
:103A5000E0916C07F0916D07FF93EF9367EF72E0D1
:103A60007F936F931F930E94990E58E250930D0419
:103A7000CDB7DEB727960FB6F894DEBF0FBECDBF29
:103A8000A0917207B0917307BF93AF9340917007F5
:103A9000509171075F934F9327E033E03F932F934B
:103AA0001F930E94990E3CE330930D048DB79EB78F
:103AB00007960FB6F8949EBF0FBE8DBFE0917607B4
:103AC000F0917707FF93EF93C0917407D09175073A
:103AD000DF93CF9387E193E02BCD10920D042BE081
:103AE00034E03F932F9311E01F930E94990EF4E16D
:103AF000F0930D040F900F900F90A0919F04B09140
:103B0000A004BF93AF93C091F903D091FA03DF9360
:103B1000CF9388E194E09F938F931F930E94990E17
:103B2000B8E2B0930D04EDB7FEB737960FB6F89430
:103B3000FEBF0FBEEDBF60919D0470919E047F9308
:103B40006F934091FB035091FC035F934F9327E2E7
:103B500034E03F932F931F930E94990E9CE3909320
:103B60000D04ADB7BEB717960FB6F894BEBF0FBE23
:103B7000ADBF8091970490919804A0919904B09161
:103B80009A04BC01CD010E94165FDC01CB019F931A
:103B90008F93C0910208D0910308DF93CF9386E3FF
:103BA00094E0C6CC10920D04CFECD4E0DF93CF9319
:103BB00011E01F930E94990E94E190930D040F90D1
:103BC0000F900F908091840399279F938F9387ED97
:103BD00094E09F938F931F930E94990E78E27093C5
:103BE0000D040F900F900F900F900F90E091DC0359
:103BF000F091DD03FF93EF9365EE74E07F936F9395
:103C00001F930E94990E5CE350930D040F900F9048
:103C10000F900F900F908091B80799279F938F93E3
:103C20008091B70799279F938F9383EF94E080CC7F
:103C300094E190930D048091A9049091AA049F931C
:103C40008F9340910104509102042091A904309176
:103C5000AA04421B530B5F934F93E5E7F3E0FF93F6
:103C6000EF93CF930E94990E78E270930D04ADB755
:103C7000BEB717960FB6F894BEBF0FBEADBF60912A
:103C8000A7047091A8047F936F934091FF03509114
:103C900000048091A7049091A804481B590B5F93DE
:103CA0004F9324E833E03F932F93CF930E94990ED4
:103CB0005CE350930D04EDB7FEB737960FB6F8945A
:103CC000FEBF0FBEEDBFA091A504B091A604BF93A7
:103CD000AF938091A5049091A6046091FD0370912B
:103CE000FE03861B970B9F938F9383E993E085CE0A
:103CF00081509C4FAF4FBF4FDBCC10920D0461E061
:103D000075E07F936F9311E01F930E94990E34E149
:103D100030930D040F900F900F90809169069927B2
:103D200087FD90959F938F9380916806992787FDD3
:103D300090959F938F9341E155E05F934F931F932D
:103D40000E94990EF8E2F0930D04EDB7FEB7379696
:103D50000FB6F894FEBF0FBEEDBF80916A0699279B
:103D600087FD90959F938F9380916B0699279F93E2
:103D70008F9321E235E03F932F931F930E94990E7A
:103D8000BCE3B0930D04ADB7BEB717960FB6F89469
:103D9000BEBF0FBEADBF80916F0699279F938F93D3
:103DA00080916C06992787FD90959F938F9381E36F
:103DB00095E0BECB81509C4FAF4FBF4FA0CC14E1DC
:103DC00010930D046BE972E07F936F9311E01F93E2
:103DD0000E94990E78E270930D040F900F900F904F
:103DE00082EA92E054CD0196FACD0196D3CD0196A8
:103DF000ACCD01962CCC019600CC0196D4CB109280
:103E00000B04DF91CF911F9108951092B9008AE2BF
:103E10008093B800089585EA8093BC0080E090E02C
:103E2000089584E98093BC0008951092B9008093AE
:103E3000BB0085E88093BC0080E090E0089564E9D1
:103E40006093BC00109212048091BB001092110488
:103E500050E85093BC001092BD001092BA0010922E
:103E6000BB001092B9001092B8001092B9004AE25B
:103E70004093B80035EA3093BC0020E02093B900AD
:103E80002093BB0085E88093BC0008951F920F9299
:103E90000FB60F9211242F933F934F935F936F931D
:103EA0007F938F939F93AF93BF93EF93FF938091F3
:103EB0001204282F3327442755278F5F809312043D
:103EC0002731310508F0D9C0F901E25CFF4FEE0F50
:103ED000FF1F0590F491E02D09941092B90080E83D
:103EE0008093BB0085E88093BC00C7C01092B900E6
:103EF00088E9F6CF74E97093BC006AE070E07093D3
:103F00009D0360939C0385EA8093BC00B6C08091BA
:103F10001004E82FFF27E25AF84F9091BB009483DA
:103F20008F5F843008F496C010921004B4E9B09307
:103F3000BC00AAE0B0E0B0939D03A0939C03109254
:103F400012049BC080911B031092B900C9CF8091CD
:103F50001104880F8E5A1092B900C2CF34E9309301
:103F6000BC0020911104243008F077C01092120494
:103F700085EACACF40911104242F33274F5F409325
:103F800011042130310509F45BC0223031050CF4F5
:103F90006FC02230310509F458C02330310509F0D3
:103FA0006CC080911C081092B9009ACF90911004B7
:103FB000E92FFF27E130F10509F442C0E230F105B5
:103FC0000CF44FC0E230F10509F43FC0339709F01B
:103FD00054C0E7CF90911004E92FFF27E25AF84F21
:103FE0005091BB005083E4CF1092B90082E178CFAA
:103FF00080911004880F8D5A1092B90071CF809172
:104000001A031092B9006CCF1092B90080E168CF0A
:104010008091100499278130910591F082309105AB
:1040200054F18230910589F0039739F5BACF809128
:1040300019031092B90054CF1092B90084E150CF07
:104040008091F8071092B9004BCF80911908109217
:10405000B90046CF8093100469CF1092110485EA0D
:1040600053CFEF2B51F48091EF071092B90038CF66
:10407000232BC9F302C0892BB1F3F091BC00F06887
:10408000F093BC00FF91EF91BF91AF919F918F9101
:104090007F916F915F914F913F912F910F900FBE44
:1040A0000F901F90189523EC2093810080916F0052
:1040B000806280936F001092A6041092A504109263
:1040C000A8041092A7041092AA041092A9040895BB
:1040D0001F920F920FB60F921124EF92FF920F933F
:1040E0001F932F933F934F935F936F937F938F9380
:1040F0009F93AF93BF93CF93DF93EF93FF93209161
:104100008600309187000091130410911404201B45
:10411000310BE0908600F0908700F0921404E0925A
:104120001304C9018D549440835F9A4180F4209117
:104130001504309116042430310514F010927F03D9
:1041400041E050E05093160440931504A1C0C09183
:104150001504D0911604CA30D1050CF099C0B901EC
:104160006B5F7040645B7140A8F0FE013196F09384
:104170001604E0931504E530F10509F469C05D9873
:10418000E630F10509F462C05C98379709F45CC029
:104190005B987EC0A901425D5140FE01EC0FFD1FFE
:1041A000EA59F84F80819181DA01A81BB90BCD0142
:1041B000B7FD6AC006972CF410914504183C08F42A
:1041C0005AC0FE01EC0FFD1FEA59F84FE080F18064
:1041D0009701220F331F2E0D3F1D240F351F37FD72
:1041E00050C07901F594E794F594E794DA011196BB
:1041F000AE15BF05BCF50894E108F10850914504DF
:10420000533C40F18E010C0F1D1FF801EA59F84F85
:1042100080819181A701481B590BCA0163E070E0BE
:104220000E9434609B01660F771F620F731F045852
:10423000184FF80171836083FE01EC0FFD1FEA59EE
:10424000F84FF182E08291CF5B9A22C05C9A9DCFB9
:104250005D9A96CFFE01EC0FFD1FE458F84F1182D6
:104260001082EACF41505040E416F5063CF608941F
:10427000E11CF11CC3CF30914504365F30934504F7
:10428000A0CF2D5F3F4FADCF909581959F4F92CF9F
:10429000FF91EF91DF91CF91BF91AF919F918F915E
:1042A0007F916F915F914F913F912F911F910F914E
:1042B000FF90EF900F900FBE0F901F90189591E018
:1042C0009093940772E07093950763E0609396076C
:1042D00054E05093970745E04093980736E03093B9
:1042E000990727E020939A0788E080939B07089519
:1042F0001F9338E630939C073EE130939D077BEF98
:1043000070939F071AE01093A00730939E07309395
:10431000A207E4E0E093A107BFE0B093A3073093C6
:10432000A4071CE01093A50778E07093A60756EE4B
:104330005093A7073093A80720E82093A90780E5AA
:104340008093AA0796E99093AB07AEE5A093AC07DC
:10435000F3E2F093AD073093AE071092AF0740E25F
:104360004093B0071092B1071092B2071092B307B2
:104370001092B4071092C4071092C5071092C60796
:104380001092C70744E64093B50768E26093B6070A
:104390001092DA0752E35093B7079093B80725E0DD
:1043A0002093B9075093BA079AE59093BB075093AF
:1043B000BC071092D9079093BD072093BE0785E5EF
:1043C0008093BF078093C007A0E1A093C107E0934B
:1043D000C2074093C307FFE5F093C80763EF6093FC
:1043E000CA07B093C907B093CB075DEF5093CC07D2
:1043F0004093CD079093CE079093CF079093D0072B
:104400001092D10726E02093D2077093D3079093A0
:10441000D4073093D5074093D6078CE38093D70712
:10442000AEE9B3E0EFEDF7E00D9001921A95E1F7F8
:104430001F9108951F9348E640939C074EE14093D7
:104440009D079BEF90939F077AE07093A00740939E
:104450009E074093A20713E01093A1071CE010935E
:10446000A30760E16093A40776E07093A50768E076
:104470006093A607B6EEB093A7074093A80780E81D
:104480008093A90750E55093AA07A8E7A093AB072C
:10449000EEE5E093AC0733E23093AD074093AE070F
:1044A0001092AF0750E25093B0071092B1071092EC
:1044B000B2071092B3071092B4071092C40710927B
:1044C000C5071092C6071092C70734E63093B507A8
:1044D000F8E2F093B6071092DA0792E39093B707E9
:1044E00026E92093B807B5E0B093B9079093BA07CF
:1044F0002AE52093BB079093BC071092D90720931D
:10450000BD07B093BE0785E58093BF078093C007C2
:104510005093C107A4E0A093C207EBE4E093C30764
:10452000FFE5F093C807B3EFB093CA0794E1909307
:10453000C9079093CB075DEF5093CC073093CD071D
:104540002093CE072093CF072093D0071092D10756
:104550007093D2076093D3072093D4074093D50775
:104560003093D6078CE38093D707A5EAB3E0EFED4D
:10457000F7E00D9001921A95E1F71F91089538EE3A
:1045800030939C073EE130939D077BEF70939F072C
:104590006AE06093A00730939E073093A20753E030
:1045A0005093A10758E05093A307F0E1F093A407BC
:1045B00066E06093A5075093A60796EE9093A70731
:1045C0003093A80740E84093A90744E64093AA0720
:1045D00028E72093AB078EE58093AC07A3E2A09376
:1045E000AD07E4E1E093AE071092AF07F093B00798
:1045F0001092B1071092B2071092B3071092B4074D
:104600001092C4071092C5071092C6071092C707F0
:104610004093B507B8E2B093B6071092DA07E2E329
:10462000E093B70776E97093B80795E09093B907E0
:10463000E093BA077AE57093BB07E093BC0710924A
:10464000D9077093BD079093BE0725E52093BF0758
:104650002093C00780E28093C107A4E0A093C20723
:10466000E093C307FFE5F093C807B3EFB093CA0721
:104670003093C9073093CB079DEF9093CC074093BD
:10468000CD077093CE077093CF077093D007109229
:10469000D1076093D2075093D3077093D407309318
:1046A000D5074093D6072CE32093D7078CE0ADEADB
:1046B000B3E0EFEDF7E00D9001928A95E1F70895F0
:1046C0000F931F93CF93C82FC150CF3F81F004E6C3
:1046D00010E080913C04882351F41093E003009390
:1046E000DF038AEF90E00E940F13C15090F7CF9143
:1046F0001F910F91089520919807E22FFF27EE0F49
:10470000FF1FEA59F84F8081918183589F4FA091F4
:104710004C04B0914D04A817B9070CF084C0CD012A
:10472000019690934D0480934C04DC0130919907DD
:10473000E32FFF27EE0FFF1FEA59F84F8081918189
:1047400083589F4F60914A0470914B046817790712
:104750000CF095C0CB01019690934B0480934A04D2
:10476000BC0150919A07E52FFF27EE0FFF1FEA5972
:10477000F84F8081918183589F4F40914804509118
:104780004904481759070CF06BC0CA010196909371
:10479000490480934804AC0190919B07E92FFF27BF
:1047A000EE0FFF1FEA59F84F8081918183589F4F88
:1047B0002091460430914704281739070CF041C076
:1047C000C901019690934704809346049C01B7FD6C
:1047D0007EC0AF3FB10511F00CF060C077FD66C040
:1047E0006F3F710539F034F06FEF70E070934B0458
:1047F00060934A0457FD60C04F3F510539F034F0D3
:10480000EFEFF0E0F0934904E093480437FD5AC01D
:104810002F3F310539F034F04FEF50E0509347040B
:104820004093460408954081518143585F4F4A1791
:104830005B070CF07BCF109709F478CFCD0101977F
:1048400070CF8081918183589F4F821793070CF01E
:10485000BECF2115310509F4BACFC9010197B2CFF6
:104860002081318123583F4F241735070CF094CF16
:104870004115510509F490CFCA01019788CF2081D5
:10488000318123583F4F261737070CF06ACF611547
:10489000710509F466CFCB0101975ECFAFEFB0E0B1
:1048A000B0934D04A0934C0477FF9ACF10924B0421
:1048B00010924A0457FFA0CF109249041092480466
:1048C00037FFA6CF10924704109246040895109225
:1048D0004D0410924C0482CF2F923F924F925F92E0
:1048E0006F927F928F929F92AF92BF92CF92DF9200
:1048F000EF92FF920F931F93CF93DF93CDB7DEB765
:1049000067970FB6F894DEBF0FBECDBFE090A50449
:10491000F090A6040091FD031091FE03E01AF10A45
:10492000F0922608E0922508A0901308B090140891
:10493000C090FD03D090FE03AC18BD08B092930761
:10494000A09292076090FF03709000048090A704EB
:104950009090A804681879087092EE076092ED07AD
:1049600040900104509002042091A9043091AA04BF
:10497000421A530A5092FA074092F90720902008F1
:104980003090210871010027F7FC0095102F8091CD
:10499000F9039091FA03AA2797FDA095BA2FBC01BD
:1049A000CD012CE030E040E050E00E94F55FDC01FA
:1049B000CB01E80EF91E0A1F1B1F17FDC0C5159578
:1049C0000795F794E794F0922108E092200840912F
:1049D0003308509134087A010027F7FC0095102F16
:1049E0008091FB039091FC03AA2797FDA095BA2F15
:1049F000BC01CD012CE030E040E050E00E94F55FCA
:104A0000DC01CB01E80EF91E0A1F1B1F17FD91C523
:104A100015950795F794E794F0923408E0923308DF
:104A200060910208709103089B01442737FD40956F
:104A3000542F8091F7039091F803AA2797FDA09532
:104A4000BA2F280F391F4A1F5B1F57FD6DC555959B
:104A50004795379527953093030820930208E090F7
:104A6000F903F090FA036CE070E0E69E5001E79ED7
:104A7000B00CF69EB00C1124C501AA2797FDA09595
:104A8000BA2F209181043091820440918304509187
:104A90008404820F931FA41FB51F809381049093F9
:104AA0008204A0938304B0938404E091FB03F0910B
:104AB000FC03E69F2001E79F500CF69F500C112449
:104AC000C201AA2797FDA095BA2F60907D0470902F
:104AD0007E0480907F0490908004860D971DA81D11
:104AE000B91D80937D0490937E04A0937F04B093BE
:104AF000800400910C0810910D084091F903509129
:104B0000FA03040F151F10930D0800930C088090F2
:104B1000280890902908C090FB03D090FC038C0CCF
:104B20009D1C9092290880922808A0919B04B09126
:104B30009C041196B0939C04A0939B0480917904EB
:104B400090917A04A0917B04B0917C04BC01CD01CA
:104B50000E94335F5B016C0180914E0790914F077B
:104B6000AA2797FDA095BA2FBC01CD010E94335F03
:104B70001B012C018091970490919804A0919904B5
:104B8000B0919A049C01AD01C201B1010E948D5EF9
:104B90009B01AC01C601B5010E948E5EDC01CB0118
:104BA000BC01CD010E94165F6093790470937A0472
:104BB00080937B0490937C04E0912508F091260873
:104BC0009F01442737FD4095542F40902F08509067
:104BD00030086090310870903208240D351D461D54
:104BE000571DA0912508B09126081D01442437FCCB
:104BF0004094542C6090610470906204809063042F
:104C000090906404260C371C481C591C29823A8257
:104C10004B825C8220926104309262044092630471
:104C200050926404283707E1300707E0400700E0AE
:104C3000500724F0285737414740504057FD6FC474
:104C400020932F0830933008409331085093320856
:104C5000109133041B87112309F09AC0309032045D
:104C6000332009F070C350909C075E8256FE93C0BB
:104C70008091920790919307AA2797FDA095BA2F4C
:104C8000209071043090720440907304509074042A
:104C90002F82388649865A86BC01CD01A201910136
:104CA0000E94F55F9B01AC0197FD6DC46BE05595CB
:104CB0004795379527956A95D1F770902504A72CCD
:104CC000BB24CC24DD24C601B5010E94F55F97FD0D
:104CD00055C43B014C019CE095948794779467946C
:104CE0009A95D1F76092AB047092AC048092AD04B7
:104CF0009092AE048091920790919307AA2797FD16
:104D0000A095BA2FE0906904F0906A0400916B04BA
:104D100010916C04BC01CD01A80197010E94F55FC0
:104D20009B01AC0197FD5AC48BE05595479537958B
:104D300027958A95D1F7C601B5010E94F55F97FDC9
:104D400048C49B01AC01BCE0559547953795279524
:104D5000BA95D1F72093AF043093B0044093B104D7
:104D60005093B204C401B30197FC2BC461387105A0
:104D7000810591054CF4CA01B90157FDF7C36138AB
:104D80007105810591055CF131E03093500427C035
:104D900090909C079E821092AF041092B0041092E3
:104DA000B1041092B2041092AB041092AC041092B1
:104DB000AD041092AE048091710490917204A091A0
:104DC0007304B09174048F839887A987BA87E090A1
:104DD0006904F0906A0400916B0410916C04A09136
:104DE000AB04B091AC048090ED079090EE07A80D55
:104DF000B91DB093EE07A093ED0750902404852DC4
:104E00009927AA27BB272091AF043091B004409185
:104E1000B1045091B204BC01CD010E94F55F9B0129
:104E2000AC0197FD14C3A9E0559547953795279593
:104E3000AA95D1F76090ED077090EE07620E731E91
:104E40007092EE076092ED076091ED077091EE07AA
:104E50003B01882477FC8094982C20916504309144
:104E600066044091670450916804620E731E841EAC
:104E7000951E6C867D868E869F864091ED075091AB
:104E8000EE07C0903604D09037044C195D095A01E2
:104E9000CC24B7FCC094DC2CAE0CBF1CC01ED11EB1
:104EA0002091920330919303409194035091950384
:104EB0002A153B054C055D0584F4F8EA6F2EF1E6F2
:104EC0007F2E812C912C621A730A840A950A640140
:104ED00053016C867D868E869F86EE24FF24870193
:104EE000E21AF30A040B150BAE14BF04C006D10678
:104EF0000CF00DC2E8E5AE2EEEE9BE2EEFEFCE2EA1
:104F0000EFEFDE2EA20EB31EC41ED51EA0926904C2
:104F1000B0926A04C0926B04D0926C0435014601D1
:104F2000A0926504B0926604C0926704D0926804AF
:104F3000E091FF03F09100043F9734F488E19CEF87
:104F40009093EE078093ED07A091FF03B0910004CA
:104F5000179734F440E358EF5093EE074093ED0772
:104F6000509101015D835A3009F45BC2E091FF0367
:104F7000F0910004E55EF7400CF0DEC1A091FF0364
:104F8000B0910004A35FB74034F040ED57E0509378
:104F9000EE074093ED072090F9073090FA07E09074
:104FA000AF04F090B0042E183F083092FA07209218
:104FB000F907852D9927AA27BB272091AB043091AB
:104FC000AC044091AD045091AE04BC01CD010E94EF
:104FD000F55F9B01AC0197FD9DC279E05595479522
:104FE000379527957A95D1F70091F9071091FA072F
:104FF000021B130B1093FA070093F9078091F9072E
:105000009091FA077C010027F7FC0095102F209162
:105010006D0430916E0440916F0450917004E20E63
:10502000F31E041F151FEC8AFD8A0E8B1F8BE09167
:10503000F907F091FA074090340450903504E419D0
:10504000F5091F01442437FC4094542C6F81788566
:1050500089859A85260E371E481E591E2C863D8648
:105060004E865F8620919603309197034091980376
:1050700050919903221533054405550594F468EAC7
:10508000E62E61E6F62E012D112DE21AF30A040B2D
:10509000150BEC86FD860E871F87EC8AFD8A0E8B2A
:1050A0001F8B88279927DC01821B930BA40BB50B60
:1050B0002C843D844E845F84281639064A065B069C
:1050C0000CF054C1285A3146404050402C873D874F
:1050D0004E875F872093710430937204409373046A
:1050E0005093740479018A0120936D0430936E0407
:1050F00040936F0450937004A0910104B091020496
:105100001F9734F4E8E1FCEFF093FA07E093F90716
:1051100020910104309102042730310534F480E3FA
:1051200098EF9093FA078093F9079D819A3009F4DC
:1051300062C1A0910104B0910204A55EB74034F0B1
:1051400028EE33E03093FA072093F90780910104A9
:1051500090910204835F974034F040ED57E0509304
:10516000FA074093F9077FEE70937A0069817A819C
:105170008B819C816093750470937604809377048F
:10518000909378042C843D844E845F842092910413
:10519000309292044092930450929404A092890415
:1051A000B0928A04C0928B04D0928C04E0928D0459
:1051B000F0928E0400938F04109390046092850403
:1051C000709286048092870490928804DE80D7FCD7
:1051D00053C110919807E12FFF27EE0FFF1FEA59E7
:1051E000F84F8081918183589F4FA0914C04B091DA
:1051F0004D04A817B9070CF0F0C0CD0101969093AB
:105200004D0480934C04DC0130909907E32DFF2777
:10521000EE0FFF1FEA59F84F0081118103581F4F0D
:1052200060914A0470914B04601771070CF0C6C07E
:10523000CB01019690934B0480934A04BC0150909B
:105240009A07E52DFF27EE0FFF1FEA59F84F8081DF
:10525000918183589F4F40914804509149044817C9
:1052600059070CF09CC0CA010196909349048093A1
:105270004804AC0170909B07E72DFF27EE0FFF1F3E
:10528000EA59F84F8081918183589F4F20914604BD
:1052900030914704281739070CF059C0C90101960D
:1052A00090934704809346049C01B7FD2EC1AF3F05
:1052B000B10539F034F0EFEFF0E0F0934D04E093F6
:1052C0004C0477FDD4C06F3F710539F034F06FEFB7
:1052D00070E070934B0460934A0457FDBDC04F3F8C
:1052E000510539F034F0AFEFB0E0B0934904A0932A
:1052F000480437FDB7C02F3F310509F00CF473C1E6
:105300004FEF50E050934704409346046CC1A09285
:105310006904B0926A04C0926B04D0926C040C854C
:105320001D852E853F8500936504109366042093A8
:10533000670430936804FCCD88EE93E09093EE0709
:105340008093ED071BCEB0909C07BE8224CD0081D8
:10535000118103581F4F021713070CF0A6CF211518
:10536000310509F4A2CFC90101979ACF6C857D85DB
:105370008E859F856093710470937204809373048B
:10538000909374044C895D896E897F8940936D0484
:1053900050936E0460936F0470937004ADCE0081DF
:1053A000118103581F4F041715070CF063CF4115E7
:1053B000510509F45FCFCA01019757CF2081318190
:1053C00023583F4F261737070CF039CF6115710569
:1053D00009F435CFCB0101972DCF4081518143583E
:1053E0005F4F4A175B070CF00FCF109709F40CCFF3
:1053F000CD01019704CF4091010450910204435F15
:10540000534034F068EE73E07093FA076093F90745
:10541000E0910104F0910204EA5FF3400CF4A3CEA2
:105420009CCE6091FF0370910004635F734034F081
:1054300028EE33E03093EE072093ED070091FF0351
:10544000109100040A5F13400CF4A5CD9ECD2150AD
:105450003E4F4F4F5F4FE7CC1092490410924804E3
:1054600037FF49CF1092470410924604BCC01092F7
:105470004B0410924A0431CFFB84FF2009F0A9CEDF
:10548000B0913204BB2309F0A4CE0091F90710912A
:10549000FA07093C11050CF058C0E091F907F091AA
:1054A000FA07E853FF4FA4F48091F9079091FA07A7
:1054B000880F991F880F991F8090F9079090FA071D
:1054C000880D991D805E9C4F9093FA078093F90791
:1054D000A091ED07B091EE07A93CB1050CF458C0BE
:1054E0008091ED079091EE07880F991F880F991F03
:1054F000C090ED07D090EE078C0D9D1D805293401B
:105500009093EE078093ED0764CE10924D041092B5
:105510004C04D7CE21503E4F4F4F5F4F5ECD2858A1
:10552000384E484F5F4F8CCB2F5F3F4F4F4F5F4FF1
:105530008ECA0894E11CF11C011D111D69CA089452
:10554000E11CF11C011D111D3ACA8091F9079091CF
:10555000FA07880F991F880F991FA090F907B0903C
:10556000FA078A0D9B1D80529340AECF909580958F
:10557000709561957F4F8F4F9F4F01CC6150704F59
:105580008F4F9F4FA6CB2150384F4F4F5F4F8ECB41
:105590002091ED073091EE0728533F4F0CF019CEC4
:1055A0008091ED079091EE07880F991F880F991F42
:1055B0006090ED077090EE07860D971D805E9C4F02
:1055C0009FCF90958095709561957F4F8F4F9F4F9E
:1055D000CDCB6150704F8F4F9F4FB3CB2150384F81
:1055E0004F4F5F4FA1CB67960FB6F894DEBF0FBE4B
:1055F000CDBFDF91CF911F910F91FF90EF90DF9082
:10560000CF90BF90AF909F908F907F906F905F9062
:105610004F903F902F900895809101018D3009F4B3
:105620003FC110927A0080910104909102049093FE
:10563000FA078093F907E091FF03F0910004F093DB
:10564000EE07E093ED07A091FD03B091FE03B09348
:105650002608A09325088091F9039091FA03AA27C0
:1056600097FDA095BA2FBC01CD012CE030E040E0C1
:1056700050E00E94F55FDC01CB01909321088093FC
:1056800020088091FB039091FC03AA2797FDA09529
:10569000BA2FBC01CD010E94F55FDC01CB019093D4
:1056A0003408809333086091F7037091F803709386
:1056B0000308609302084FEE40937A0030919807F8
:1056C000E32FFF27EE0FFF1FEA59F84F20813181AA
:1056D00023583F4FA0914C04B0914D04A217B3073B
:1056E0000CF085C0CD01019690934D0480934C043D
:1056F000DC0150919907E52FFF27EE0FFF1FEA59B4
:10570000F84F4081518143585F4F60914A04709136
:105710004B04641775070CF096C0CB01019690936B
:105720004B0480934A04BC0190919A07E92FFF270C
:10573000EE0FFF1FEA59F84F2081318123583F4F68
:105740004091480450914904421753070CF06CC033
:10575000CA0101969093490480934804AC013091AA
:105760009B07E32FFF27EE0FFF1FEA59F84F8081B9
:10577000918183589F4F2091460430914704281708
:1057800039070CF042C0C9010196909347048093F9
:1057900046049C01B7FD7FC0AF3FB10511F00CF08E
:1057A00061C077FD67C06F3F710539F034F06FEF6E
:1057B00070E070934B0460934A0457FD61C04F3F03
:1057C000510539F034F0EFEFF0E0F0934904E09345
:1057D000480437FD5BC02F3F310509F00CF463C06E
:1057E0004FEF50E050934704409346045CC0208143
:1057F000318123583F4F2A173B070CF07ACF10977F
:1058000009F477CFCD0101976FCF808191818358C3
:105810009F4F821793070CF0BDCF2115310509F476
:10582000B9CFC9010197B1CF8081918183589F4F32
:10583000841795070CF093CF4115510509F48FCFCC
:10584000CA01019787CF8081918183589F4F861726
:1058500097070CF069CF6115710509F465CFCB018D
:1058600001975DCFAFEFB0E0B0934D04A0934C042F
:1058700077FF99CF10924B0410924A0457FF9FCFA5
:10588000109249041092480437FFA5CF10924704A4
:105890001092460408C010924D0410924C0481CF1F
:1058A0000E94D214BECE8091BF079927AA27BB279A
:1058B000BC01CD0124EC39E040E050E00E94F55FEE
:1058C000DC01CB018093960390939703A0939803F8
:1058D000B09399038091C0079927AA27BB27BC01E1
:1058E000CD010E94F55F60939203709393038093C0
:1058F00094039093950308951092A00410929F042E
:1059000010929E0410929D0420E030E040E050E0B0
:1059100020939704309398044093990450939A04E9
:105920001092AA041092A9041092A8041092A7043D
:105930001092A6041092A504109214081092130855
:1059400010922504109224041092F003809101011A
:105950008D3009F476C310927A0080910104909101
:1059600002049093FA078093F907E091FF03F09106
:105970000004F093EE07E093ED07A091FD03B091D2
:10598000FE03B0932608A09325088091F903909117
:10599000FA03AA2797FDA095BA2FBC01CD012CE0F0
:1059A00030E040E050E00E94F55FDC01CB019093D5
:1059B0002108809320088091FB039091FC03AA2783
:1059C00097FDA095BA2FBC01CD010E94F55FDC01C7
:1059D000CB0190933408809333086091F703709162
:1059E000F80370930308609302085FEE50937A0007
:1059F00030919807E32FFF27EE0FFF1FEA59F84F6A
:105A00004081518143585F4FA0914C04B0914D04A7
:105A1000A417B5070CF02BC2CD01019690934D044D
:105A200080934C04DC0170919907E72FFF27EE0F5C
:105A3000FF1FEA59F84F4081518143585F4F6091F1
:105A40004A0470914B04641775070CF03CC2CB01FB
:105A5000019690934B0480934A04BC0190919A075D
:105A6000E92FFF27EE0FFF1FEA59F84F2081318100
:105A700023583F4F4091480450914904421753071F
:105A80000CF012C2CA010196909349048093480415
:105A9000AC0130919B07E32FFF27EE0FFF1FEA5960
:105AA000F84F8081918183589F4F20914604309117
:105AB0004704281739070CF0E8C1C90101969093F3
:105AC0004704809346049C01B7FDB0C2AF3FB105C7
:105AD00011F00CF007C277FD0DC26F3F710539F070
:105AE00034F06FEF70E070934B0460934A0457FDFD
:105AF00007C24F3F510539F034F0EFEFF0E0F0937B
:105B00004904E093480437FD01C22F3F310539F0C5
:105B100034F04FEF50E05093470440934604809197
:105B2000BF079927AA27BB27BC01CD0124EC39E088
:105B300040E050E00E94F55FDC01CB0180939603CA
:105B400090939703A0939803B09399038091C00713
:105B50009927AA27BB27BC01CD010E94F55F60935E
:105B6000920370939303809394039093950384E638
:105B700090E00E942113B0910101BD3009F45EC292
:105B800010927A0020910104309102043093FA07B8
:105B90002093F9074091FF03509100045093EE07C2
:105BA0004093ED07E091FD03F091FE03F09326088A
:105BB000E09325088091F9039091FA03AA2797FDB5
:105BC000A095BA2FBC01CD012CE030E040E050E0C0
:105BD0000E94F55FDC01CB0190932108809320089F
:105BE0008091FB039091FC03AA2797FDA095BA2F03
:105BF000BC01CD010E94F55FDC01CB01909334081C
:105C000080933308A091F703B091F803B093030891
:105C1000A0930208FFEEF0937A0050919807E52FC9
:105C2000FF27EE0FFF1FEA59F84F6081718163581B
:105C30007F4FA0914C04B0914D04A617B7070CF00C
:105C400088C1CD01019690934D0480934C04DC01F2
:105C500070919907E72FFF27EE0FFF1FEA59F84FC2
:105C60004081518143585F4F60914A0470914B04C9
:105C7000641775070CF05EC1CB01019690934B043D
:105C800080934A04BC0190919A07E92FFF27EE0FF9
:105C9000FF1FEA59F84F8081918183589F4F4091AF
:105CA000480450914904481759070CF060C1CA01D3
:105CB00001969093490480934804AC0130919B076E
:105CC000E32FFF27EE0FFF1FEA59F84F80819181E4
:105CD00083589F4F20914604309147042817390775
:105CE0000CF019C1C90101969093470480934604B2
:105CF0009C01B7FD96C1AF3FB10539F034F0AFEF6D
:105D0000B0E0B0934D04A0934C0477FD79C16F3F90
:105D1000710539F034F06FEF70E070934B046093CD
:105D20004A0457FD73C14F3F510539F034F0EFEF8E
:105D3000F0E0F0934904E093480437FD6DC12F3F34
:105D4000310539F034F04FEF50E050934704409361
:105D500046048091BF079927AA27BB27BC01CD0124
:105D600024EC39E040E050E00E94F55FDC01CB011B
:105D70008093960390939703A0939803B09399030D
:105D80008091C0079927AA27BB27BC01CD010E949B
:105D9000F55F6093920370939303809394039093C1
:105DA0009503B0919C07B0FF10C0A0911C03B09167
:105DB0001D03A75BB34008F03EC160911C037091C6
:105DC0001D036E5E724008F436C1E0910104F0914B
:105DD0000204F093AA04E093A9044091FF035091B8
:105DE00000045093A8044093A7048091FD03909170
:105DF000FE039093A6048093A5042091FD033091A7
:105E0000FE0330931408209313085093A404409386
:105E1000A304F093A204E093A10444E050E0DA016B
:105E20000E948460F02DF53008F4B0C080913308F2
:105E30009091340897FD0CC16CE070E00E943460D2
:105E400070939E0460939D04809120089091210896
:105E500097FDFAC06CE070E00E9434607093A0047B
:105E600060939F0480914E0790914F07F5C0208169
:105E7000318123583F4F2A173B070CF0D4CD1097A0
:105E800009F4D1CDCD010197C9CD8081918183588D
:105E90009F4F821793070CF017CE2115310509F497
:105EA00013CEC90101970BCE8081918183589F4FFA
:105EB000841795070CF0EDCD4115510509F4E9CD96
:105EC000CA010197E1CD8081918183589F4F861748
:105ED00097070CF0C3CD6115710509F4BFCDCB0157
:105EE0000197B7CDAFEFB0E0B0934D04A0934C0451
:105EF00077FFF3CD10924B0410924A0457FFF9CD6F
:105F0000109249041092480437FFFFCD10924704C5
:105F10001092460404CE8081918183589F4F82174E
:105F200093070CF0E6CE2115310509F4E2CEC90144
:105F30000197DACE2081318123583F4F261737074A
:105F40000CF0A1CE6115710509F49DCECB0101972E
:105F500095CE8081918183589F4F8A179B070CF0C3
:105F600077CE109709F474CECD0101976CCE2081C5
:105F7000318123583F4F241735070CF09FCE411530
:105F8000510509F49BCECA01019793CEDA010E9414
:105F90008460802D9927982F88274F5F5F4FDA0103
:105FA0000E948460702D870F911D9093A0048093B0
:105FB0009F044F5F5F4FDA010E948460802D992714
:105FC000782F66274F5F5F4FDA010E948460302D83
:105FD000630F711D70939E0460939D044F5F5F4F2C
:105FE000DA010E948460802D9927982F88274F5FBF
:105FF0005F4FDA010E948460502D850F911D2CC0E7
:1060000010924B0410924A0457FF8DCE109249040F
:106010001092480437FF93CE109247041092460422
:1060200098CE10924D0410924C046FCE10924D04F5
:1060300010924C0450CD0E948014C7CE0E94D214FE
:106040009FCD0E94D21487CC909581959F4F02CF0F
:10605000909581959F4FF0CEAA2797FDA095BA2FD6
:10606000BC01CD010E94335F609397047093980444
:106070008093990490939A04109271041092720480
:10608000109273041092740410926D0410926E04B6
:1060900010926F04109270041092690410926A04B6
:1060A00010926B0410926C041092650410926604B6
:1060B00010926704109268041092610410926204B6
:1060C00010926304109264041092FA071092F90778
:1060D0001092EE071092ED071092260810922508F4
:1060E00084E690E00E94211380911E0390911F038B
:1060F000A0912003B0912103909351078093500702
:106100001092EF031092EE031092590410925A0469
:1061100010925B0410925C046091570470915804D3
:1061200070935604609355040E949756E2E3F0E0A2
:10613000F093E003E093DF038091BF079927AA273C
:10614000BB27BC01CD0124EC39E040E050E00E94C7
:10615000F55FDC01CB018856954CAF4FBF4F809364
:10616000960390939703A0939803B093990380911B
:10617000C0079927AA27BB27BC01CD010E94F55F64
:10618000DC01CB018856954CAF4FBF4F80939203F3
:1061900090939303A0939403B0939503109281037B
:1061A000109280038091570490915804AA2797FD7C
:1061B000A095BA2FBC01CD012BE035E040E050E0C6
:1061C0000E94F55F60932F08709330088093310828
:1061D0009093320810924F0410924E0441E0409385
:1061E00000010E944A5AF0911704F460F0931704DA
:1061F000BFEFB0939C088091C20799278295929532
:10620000907F9827807F982780939D0890E29093B5
:106210009E08089580913C04882321F02091C707AF
:1062200023FF25C01092F8071092EF07109219086B
:1062300010921C088091C0038823B1F48091C1039F
:10624000882311F08093F8078091C203882311F00E
:1062500080931C088091C303882311F08093190850
:10626000809117048C7F06C08093EF07E7CF809161
:1062700017048160809317048091EF07992790930A
:106280002307809322078091F80799279093250789
:106290008093240780911C08992790932707809367
:1062A000260780911908992790932907809328073A
:1062B00010921204109211040E940B1F0895CF93A4
:1062C00080919F078B3F68F08B3F09F46FC28C3F32
:1062D00009F4FCC28D3F09F484C28E3F21F4809101
:1062E000460480938C0380919E078B3F08F4DCC1A9
:1062F0008B3F09F4D7C18C3F09F4FDC28D3F09F4EF
:1063000088C28E3F09F409C380918D03882309F068
:10631000D0C180938D038091A0078B3F08F4D0C13A
:106320008B3F09F4CBC18C3F09F4D3C28D3F09F4F4
:1063300073C28E3F09F4E5C280918B03882309F074
:10634000C4C180938B038091A2078B3F68F08B3F81
:1063500009F43EC28C3F09F4AAC28D3F09F444C23D
:106360008E3F21F48091460480938A038091A9078F
:106370008B3F68F08B3F09F42EC28C3F09F4A3C217
:106380008D3F09F42BC28E3F21F480914604809307
:1063900089038091AA078B3F08F49EC18B3F09F4C3
:1063A00099C18C3F09F48CC28D3F09F426C28E3FFF
:1063B00009F4ADC2809188038B3008F492C18F3FFD
:1063C00011F4809388038091AB078B3F68F08B3F7B
:1063D00009F4FBC18C3F09F46DC28D3F09F410C272
:1063E0008E3F21F480914604809387038091B0070B
:1063F0008B3F08F478C18B3F09F4E1C18C3F09F46D
:106400005CC28D3F09F4F6C18E3F09F477C2C0919A
:1064100085038091B1078B3F08F06DC180932D04F7
:106420008091B2078B3F68F08B3F09F4C2C18C3F6B
:1064300009F45EC28D3F09F4E9C18E3F21F48091D9
:10644000460480932C048091B3078B3F68F08B3F08
:1064500009F4B2C18C3F09F427C28D3F09F4C7C1CA
:106460008E3F21F48091460480932B048091B407E1
:106470008B3F68F08B3F09F493C18C3F09F411C244
:106480008D3F09F4E4C18E3F21F48091460480934E
:106490002A048091C4078B3F08F43EC18B3F09F466
:1064A00039C18C3F09F4E8C18D3F09F4D3C18E3F57
:1064B00009F430C280910408882309F032C1809326
:1064C00004088091C5078B3F08F432C18B3F09F463
:1064D0002DC18C3F09F4D6C18D3F09F4BEC18E3F5A
:1064E00009F421C280910708882309F026C180930E
:1064F00007088091C6078B3F68F08B3F09F44DC1B8
:106500008C3F09F4B6C18D3F09F4AAC18E3F21F436
:1065100080914604809327048091C7078B3F68F0E1
:106520008B3F09F440C18C3F09F4A0C18D3F09F4B1
:106530009AC18E3F21F48091460480932604809175
:10654000B5078B3F68F08B3F09F41BC18C3F09F402
:106550009CC18D3F09F478C18E3F21F4809146049F
:10656000809384038091BA078B3F68F08B3F09F4D6
:106570000BC18C3F09F48CC18D3F09F45CC18E3F87
:1065800021F480914604809383038091BD078B3F63
:1065900068F08B3F09F4EFC08C3F09F49DC18D3F3B
:1065A00009F446C18E3F21F480914604809325046E
:1065B0008091BE078B3F68F08B3F09F4DFC08C3FB2
:1065C00009F469C18D3F09F42AC18E3F21F48091FD
:1065D0004604809324048091C3078B3F68F08B3F6F
:1065E00009F4D8C08C3F09F44AC18D3F09F41AC19F
:1065F0008E3F21F480914604809382038091C907E5
:106600008B3F08F4A1C08B3F09F49CC08C3F09F478
:1066100045C18D3F09F412C18E3F09F481C18091BB
:106620000E08823008F495C08F3F11F480930E0855
:106630008091CB078B3F08F490C08B3F09F48BC04F
:106640008C3F09F44FC18D3F09F4FBC08E3F09F424
:106650005BC180912308823008F484C08F3F11F41D
:10666000809323088091D8078B3F68F08B3F09F413
:106670008EC08C3F09F433C18D3F09F4D6C08E3FE4
:1066800021F480914604809336088C2F992787FD4A
:106690009095A92FB92FBC01CD010E94335FC7FF90
:1066A00045C162C080914C0480938D03882309F416
:1066B00030CE843608F42FCE84E62BCE80914C0465
:1066C00080938B03882309F43CCE843608F43BCEB8
:1066D00084E637CE80914C04809388038B3008F099
:1066E0006ECE8AE06ECEC82FC09385038091B1072D
:1066F0008B3F08F493CE8B3F09F464C08C3F09F4C0
:10670000F4C08D3F09F47FC08E3F09F089CE80919F
:10671000460484CE80914C0480930408882309F4B5
:10672000CECE8A3F08F4CDCE8AEFC9CE80914C04FC
:1067300080930708882309F4DACE8A3F08F4D9CE7B
:106740008AEFD5CE80914C0480930E08823008F0F9
:106750006BCF81E06BCF80914C0480932308823013
:1067600008F07CCF81E07CCF20E030E040E853E4CB
:106770000E948E5EDBC080914C0418CF80914C0447
:1067800028CF80914C04ECCE80914C04FCCE8091BB
:106790004C0479CF80914C042FCF80914C04BACE19
:1067A00080914C0474CE80914C04C7CE80914C04EF
:1067B00098CD80914C0445CE80914C0455CEC0912B
:1067C0004C0492CF80914C0429CE80914C040CCE85
:1067D00080914C04C9CD80914C04D9CD809148045E
:1067E000D6CD809148047DCD80914804BDCD809167
:1067F00048043ACEC091480477CF809148046CCFCA
:1068000080914804F1CD8091480408CE80914804DD
:1068100018CE8091480448CF8091480451CF809190
:106820004804D7CE80914804E7CE809148042BCF0E
:1068300080914804BBCE80914804A5CE8091480445
:1068400083CF8091480489CF8091480489CE80917C
:1068500048041DCE809148045FCF8091480468CFE2
:106860008091480457CE8091480467CE80914A04B5
:1068700064CE80914A044ECE80914A044DCF8091DF
:106880004A04BACE80914A0453CF80914A0468CE1C
:1068900080914A0478CE80914A049BCE80914A042C
:1068A00053CF80914A04F3CD80914A04DDCD80918D
:1068B0004A045ACD80914A0497CDC0914A0414CF1E
:1068C00080914A0409CF80914A0461CD80914A04A5
:1068D00008CD80914A04F4CE80914A0467CE80911D
:1068E0004A04D1CE80914A0438CF80914A0496CD93
:1068F00080914A04A6CD80914A04D6CEC091460428
:10690000F3CE80914604DCCE8091460426CF809160
:106910004604E2CE80914604FFCE80914604C4CE68
:106920008091460411CF8091460402CF27E137EBD6
:1069300041ED58E30E94AD5FDC01CB0180938E03F3
:1069400090938F03A0939003B09391032091A70796
:10695000209324088091A6078093FC07CF91089587
:106960002F923F924F925F926F927F928F929F925F
:10697000AF92BF92CF92DF92EF92FF920F931F934D
:10698000CF93DF93CDB7DEB7C055D0400FB6F894A4
:10699000DEBF0FBECDBFE090A504F090A60400912D
:1069A000FD031091FE03E01AF10AF0922608E0922E
:1069B0002508A0901308B0901408C090FD03D09053
:1069C000FE03AC18BD08B0929307A09292076090A6
:1069D000FF03709000048090A7049090A8046818AA
:1069E00079087092EE076092ED0740900104509094
:1069F00002042091A9043091AA04421A530A509229
:106A0000FA074092F9072090200830902108710180
:106A10000027F7FC0095102F8091F9039091FA035D
:106A2000AA2797FDA095BA2FBC01CD012CE030E03C
:106A300040E050E00E94F55FDC01CB01E80EF91E5A
:106A40000A1F1B1F17FF02C00C94254D15950795B3
:106A5000F794E794F0922108E092200840913308DF
:106A6000509134087A010027F7FC0095102F80918F
:106A7000FB039091FC03AA2797FDA095BA2FBC01B8
:106A8000CD012CE030E040E050E00E94F55FDC01F9
:106A9000CB01E80EF91E0A1F1B1F17FF02C00C9442
:106AA0001E4D15950795F794E794F0923408E092FF
:106AB000330860910208709103089B01442737FD59
:106AC0004095542F8091F7039091F803AA2797FDE2
:106AD000A095BA2F280F391F4A1F5B1F57FF02C00E
:106AE0000C94184D55954795379527953093030885
:106AF00020930208A090F903B090FA036CE070E0D4
:106B0000A69E3001A79E700CB69E700C1124C30186
:106B1000AA2797FDA095BA2F209181043091820475
:106B20004091830450918404820F931FA41FB51FCA
:106B30008093810490938204A0938304B09384048F
:106B4000A091FB03B091FC03A69F2001A79F500CCE
:106B5000B69F500C1124C201AA2797FDA095BA2F09
:106B600020907D0430907E0440907F0450908004FB
:106B7000820D931DA41DB51D80937D0490937E040A
:106B8000A0937F04B093800400910C0810910D082D
:106B90004091F9035091FA03040F151F10930D084B
:106BA00000930C088090280890902908C090FB035F
:106BB000D090FC038C0C9D1C909229088092280890
:106BC000E0919B04F0919C043196F0939C04E09337
:106BD0009B048091790490917A04A0917B04B091F8
:106BE0007C04BC01CD010E94335F3B014C018091CC
:106BF0004E0790914F07AA2797FDA095BA2FBC0189
:106C0000CD010E94335F7B018C01809197049091AC
:106C10009804A0919904B0919A049C01AD01C80117
:106C2000B7010E948D5E9B01AC01C401B3010E94BB
:106C30008E5EDC01CB01BC01CD010E94165F60932A
:106C4000790470937A0480937B0490937C04A091E0
:106C50002508B09126087D010027F7FC0095102F2C
:106C600040902F08509030086090310870903208A2
:106C7000E40CF51C061D171D80912508909126082F
:106C8000AA2797FDA095BA2F209061043090620446
:106C90004090630450906404820D931DA41DB51DA3
:106CA0008093610490936204A0936304B09364049E
:106CB00028E7E21627E1F20627E0020720E01207A4
:106CC00044F088E898EEA8EFBFEFE80EF91E0A1F1F
:106CD0001B1F17FF02C00C940B4DE0922F08F0927F
:106CE00030080093310810933208B0903304BF820B
:106CF000BB2009F0A6C030903204332009F037C61B
:106D000050909C075A8656FE9FC0809192079091A2
:106D10009307AA2797FDA095BA2FE0907104F090F1
:106D200072040091730410917404EA8EFB8E0C8F30
:106D30001D8FBC01CD01A80197010E94F55F9B0149
:106D4000AC0197FF02C00C949054EBE05595479529
:106D500037952795EA95D1F770902504A72CBB2489
:106D6000CC24DD24C601B5010E94F55F97FF02C067
:106D70000C948A543B014C017CE095948794779461
:106D800067947A95D1F76092AB047092AC048092CC
:106D9000AD049092AE048091920790919307AA2738
:106DA00097FDA095BA2FE0906904F0906A040091D5
:106DB0006B0410916C04BC01CD01A80197010E94E5
:106DC000F55F9B01AC0197FF02C00C94B3546BE0DC
:106DD00055954795379527956A95D1F7C601B50121
:106DE0000E94F55F97FF02C00C94AD549B01AC016B
:106DF0009CE055954795379527959A95D1F720931F
:106E0000AF043093B0044093B1045093B204C40172
:106E1000B30197FE02C00C9481546138710581055D
:106E200091055CF4CA01B90157FF02C00C943554B6
:106E300061387105810591055CF131E030935004B2
:106E400027C0F0909C07FA861092AF041092B0040D
:106E50001092B1041092B2041092AB041092AC04E0
:106E60001092AD041092AE04809071049090720460
:106E7000A0907304B09074048A8E9B8EAC8EBD8EED
:106E8000E0906904F0906A0400916B0410916C0426
:106E9000E091AB04F091AC04C090ED07D090EE0708
:106EA000EC0DFD1DF093EE07E093ED0790902404A8
:106EB000892D9927AA27BB272091AF043091B004D0
:106EC0004091B1045091B204BC01CD010E94F55F24
:106ED0009B01AC0197FF02C00C945A4D89E0559577
:106EE0004795379527958A95D1F7A091ED07B091F1
:106EF000EE07A20FB31FB093EE07A093ED076091CA
:106F0000ED077091EE075B01CC24B7FCC094DC2C3C
:106F10004090650450906604609067047090680427
:106F2000A40CB51CC61CD71C2D96ACAEBDAECEAE07
:106F3000DFAE2D978091ED079091EE0720903604FB
:106F40003090370482199309AA2797FDA095BA2F8C
:106F50008E0D9F1DA01FB11F2091920330919303AE
:106F60004091940350919503281739074A075B070E
:106F70000CF0EDC488EA91E6A0E0B0E0821B930B30
:106F8000A40BB50B8093690490936A04A0936B04DF
:106F9000B0936C045C016D012D968CAF9DAFAEAFCC
:106FA000BFAF2D97EE24FF248701E21AF30A040BEA
:106FB000150B2090690430906A0440906B04509047
:106FC0006C042E143F04400651060CF0B1C4DA01E3
:106FD000C901885A9146A040B040809369049093BB
:106FE0006A04A0936B04B0936C045C016D01809300
:106FF000650490936604A0936704B09368041C0131
:107000002D012091FF03309100042F30310534F41D
:1070100048E15CEF5093EE074093ED07E091FF03EA
:10702000F0910004379734F460E378EF7093EE0743
:107030006093ED07909101019B879A3011F40C94B5
:10704000CD4A2091FF0330910004255E37400CF0BB
:1070500087C46091FF0370910004635F774034F050
:10706000E0EDF7E0F093EE07E093ED076090F907AD
:107070007090FA07E090AF04F090B0046E187F08AB
:107080007092FA076092F907892D9927AA27BB27E2
:107090002091AB043091AC044091AD045091AE040A
:1070A000BC01CD010E94F55F9B01AC0197FF02C0BE
:1070B0000C942C4D19E055954795379527951A95C1
:1070C000D1F74091F9075091FA07421B530B5093A7
:1070D000FA074093F9078090F9079090FA07940116
:1070E000442737FD4095542F80916D0490916E0494
:1070F000A0916F04B0917004280F391F4A1F5B1FC5
:107100002D962CAF3DAF4EAF5FAF2D9739014A01A1
:107110008091F9079091FA07A0913404B091350459
:107120008A1B9B0BAA2797FDA095BA2F0A8D1B8D52
:107130002C8D3D8D800F911FA21FB31F20919603B0
:10714000309197034091980350919903281739077C
:107150004A075B070CF0F8C588EA91E6A0E0B0E0CA
:10716000821B930BA40BB50B809371049093720454
:10717000A0937304B09374042D968CAF9DAFAEAF03
:10718000BFAF2D973C014D0188279927DC01821B59
:10719000930BA40BB50BE0907104F0907204009176
:1071A000730410917404E816F9060A071B070CF023
:1071B000C2C5DA01C901885A9146A040B040809307
:1071C000710490937204A0937304B09374042D9689
:1071D0008CAF9DAFAEAFBFAF2D9780936D049093F2
:1071E0006E04A0936F04B09370047C018D016091D4
:1071F0000104709102046F30710534F4E8E1FCEF92
:10720000F093FA07E093F907A0910104B09102040A
:10721000179734F420E338EF3093FA072093F907F7
:107220005B855A3011F40C94E54AE0910104F09129
:107230000204E55EF74034F0A8EEB3E0B093FA073D
:10724000A093F9072091010430910204235F374095
:1072500034F040ED57E05093FA074093F9077FEE82
:1072600070937A006090610470906204809063046F
:107270009090640460927504709276048092770412
:1072800090927804E0929104F09292040093930417
:10729000109394042092890430928A0440928B04C3
:1072A00050928C042D962CAC3DAC4EAC5FAC2D971F
:1072B00020928D0430928E0440928F04509290045C
:1072C000A0928504B0928604C0928704D09288046C
:1072D000DA84D7FE02C00C94604DB0909807EB2D75
:1072E000FF27EE0FFF1FEA59F84F20813181235805
:1072F0003F4FA0914C04B0914D04A217B3070CF07E
:107300003BC5CD01019690934D0480934C04DC0164
:1073100030909907E32DFF27EE0FFF1FEA59F84F32
:107320000081118103581F4F60914A0470914B04F2
:10733000601771070CF011C5CB01019690934B04B7
:1073400080934A04BC0150909A07E52DFF27EE0F69
:10735000FF1FEA59F84F2081318123583F4F409158
:10736000480450914904421753070CF022C5CA0142
:1073700001969093490480934804AC0170909B0758
:10738000E72DFF27EE0FFF1FEA59F84F808191810B
:1073900083589F4F2091460430914704281739079E
:1073A0000CF0F8C4C90101969093470480934604F9
:1073B0009C01B7FF02C00C94544DAF3FB10539F0AA
:1073C00034F0EFEFF0E0F0934D04E0934C0477FFDE
:1073D00002C00C943E4D6F3F710539F034F06FEFF1
:1073E00070E070934B0460934A0457FF02C00C9402
:1073F000464D4F3F510539F034F0AFEFB0E0B09358
:107400004904A093480437FF02C00C944E4D2F3F0F
:10741000310539F034F04FEF50E05093470440937A
:107420004604FB85FC3008F0D3C4299A80903D04C3
:1074300090903E049A8289828091FC0799270A964F
:107440008816990614F49A8389833091450434365A
:1074500008F091C2F0900E03FF2049F4209111032F
:10746000309112032F5F3F4F11F40C948A52809198
:10747000CF049091D004009711F40C94E34C019741
:107480009093D0048093CF041B851A3011F40C9490
:10749000EC4C143111F40C94EC4C2898E091180445
:1074A000F0911904E95EF34010F40C94F64CD0907E
:1074B000AD072D2C33243A82298271E07093520457
:1074C00050919407A52FBB27AA0FBB1FFD01E458BD
:1074D000F84F1182108290919507692F7727660FD8
:1074E000771FAB014458584FFA0111821082AA59F4
:1074F000B84F11961C921E926A59784FDB01119673
:107500001C921E9290909707E92DFF27EE0FFF1F08
:10751000EA59F84F11821082F0917F03F150F093F5
:107520007F03B0917F03BF3F31F0F0905204F886A3
:10753000FF2009F44FC40E945F31C0909407CFAA86
:10754000EC2DFF27EE0FFF1FEA59F84F6080718086
:1075500073010027F7FC0095102F9090950798AEC7
:10756000A92DBB27AA0FBB1FAA59B84FAD90BC903D
:107570003501882477FC8094982CD090C707D0FEE2
:1075800066C0C801B7012FE93BE140E050E00E942E
:10759000F55F5B016C01C401B30121E634EE4FEFEE
:1075A0005FEF0E94F55F7B018C01D601C5018E194A
:1075B0009F09A00BB10BBC01CD0120E137E240E0F7
:1075C00050E00E9469602901D801C7018A0D9B1D06
:1075D000AC1DBD1DBC01CD0120E137E240E050E013
:1075E0000E946960DA01C90172010027F7FC009569
:1075F000102F909581959F4F3C01882477FC8094B3
:10760000982C8EE7E816F1040105110514F00C948E
:10761000314E93E8E9169FEFF9069FEF09079FEFB8
:10762000190744F423E8E22E2FEFF22E2FEF022F5A
:107630002FEF122FAEE76A1671048104910414F43F
:107640000C943E4E9DE7692E712C812C912C8091DB
:10765000E0049091E104AA2797FDA095BA2FB80104
:10766000A701481B590B6A0B7B0BCB01BA0123E026
:1076700030E040E050E00E946960DA01C901880F03
:10768000991FAA1FBB1F820F931FA41FB51F6C0158
:107690008091E2049091E304AA2797FDA095BA2F68
:1076A00013012401281A390A4A0A5B0AC201B101EE
:1076B00023E030E040E050E00E946960DA01C90157
:1076C000880F991FAA1FBB1F820F931FA41FB51FEE
:1076D000BC01F092E104E092E0047092E304609255
:1076E000E2048090E4049090E5049401220F331F9B
:1076F000280D391DB090A3074B2C55244E9CC0017A
:107700004F9C900D5E9C900D1124280F391F37FF60
:1077100002C00C94D0523595279535952795309019
:10772000A407432D55274C9DF0014D9DF00D5C9D08
:10773000F00D1124E20FF31FF093E504E093E4044D
:1077400020910C0530910D05E21BF30BFEABEDAB68
:10775000A091E604B091E7049D01220F331F2A0F88
:107760003B1F469C8001479C100D569C100D112418
:10777000200F311F37FF02C00C94CC52359527954E
:1077800035952795469F6001479FD00C569FD00C9A
:107790001124C20ED31ED092E704C092E604A0903A
:1077A0000A05B0900B05CA18DB08DCAACBAA909199
:1077B0009707E92FFF27EE0FFF1FEA59F84F608068
:1077C0007180222433242618370830919607E32F3E
:1077D000FF27EE0FFF1FEA59F84F6081718168584B
:1077E0007F4F2B967FAF6EAF2B9770908803872DBE
:1077F000992787FD9095A92FB92FBC01CD010E9433
:10780000335F77FE02C00C94C45220E030E040E2C7
:1078100051E40E948E5EDC01CB0120E030E040E8C4
:107820005CE3BC01CD010E94AD5F3B014C011091B6
:107830008703812F992787FD9095A92FB92FBC0128
:10784000CD010E94335F17FF02C00C94D45220E098
:1078500030EE4BE256E40E94D05E7B018C015B016E
:107860006C0150916F0650FD02C00C94FD4A70915E
:107870003608713810F40C940E4E809168069927E2
:1078800087FD9095849DA001859D500D949D500D80
:107890001124FA018DA99EA9E80FF91FF093440461
:1078A000E093430480916906992787FD9095849D14
:1078B000B001859D700D949D700D1124DB012BA9E5
:1078C0003CA9A20FB31FB0934204A093410480913E
:1078D0006A06992787FD9095820D931D9093400429
:1078E00080933F0450906C06452D552747FD5095D9
:1078F0008091A1079927489F1001499F300C589FFC
:10790000300C1124309281032092800380916B0609
:1079100099272B964EAC5FAC2B978415950514F0E8
:107920000C94DF5290933E0480933D040C94154BCD
:107930002D960CAD1DAD2EAD3FAD2D97009365047A
:107940001093660420936704309368045ACB8093A5
:10795000690490936A04A0936B04B0936C0422CBE7
:1079600048EE53E05093EE074093ED0772CB9090B2
:107970009C079A8669CA109145041D3808F4CCCD3D
:10798000109252049091AE0782E3989F3001112427
:107990007092D0046092CF0429813A812932310556
:1079A00014F00C94695280911804909119048F3F3F
:1079B000910519F010F00C94BD521092B30410927E
:1079C000B4041092B5041092B6041092B704109249
:1079D000B8041092B9041092BA048A3F910511F4C8
:1079E0000C94515420919607E22FFF27EE0FFF1FB2
:1079F000EA59F84F80819181813591050CF4EAC0F4
:107A000030913C04332309F0E5C0A0909707EA2D9C
:107A1000FF27EE0FFF1FEA59F84F008111810C3448
:107A2000110514F40C9479538091D1048F5F893C33
:107A300010F40C9456556B856C3010F00C94F55581
:107A4000299810923C041092D104109219041092BB
:107A5000180430919407E32FFF27EE0FFF1FEA5918
:107A6000F84FA081B181A734B10514F00C94F855FA
:107A700020919507E22FFF27EE0FFF1FEA59F84FDD
:107A8000808191810190F081E02DF7FF02C00C947C
:107A90006D56E734F1050CF470C041E0A22FBB270E
:107AA000AA0FBB1FAA59B84F8D919C91119787348B
:107AB000910544F0E32FFF27EE0FFF1FEA59F84F1F
:107AC000808191810D911C910734110564F0E32FA1
:107AD000FF27EE0FFF1FEA59F84F6081718167346D
:107AE00071050CF042E0E22FFF27EE0FFF1FEA596D
:107AF000F84FA081B181A634B10564F4E32FFF27CC
:107B0000EE0FFF1FEA59F84F80819181873491056C
:107B10000CF043E0E22FFF27EE0FFF1FEA59F84F6A
:107B2000608171816A5B7F4F64F4E32FFF27EE0F62
:107B3000FF1FEA59F84F00811181073411050CF03D
:107B400044E0E22FFF27EE0FFF1FEA59F84FA08114
:107B5000B181AA5BBF4F64F4E32FFF27EE0FFF1F35
:107B6000EA59F84F20813181263431050CF445E083
:107B7000842F0E94E60220919507E22FFF27EE0F47
:107B8000FF1FEA59F84F808191810190F081E02D2B
:107B9000F7FF02C00C9402567E9714F00C94A35584
:107BA000C0909407EC2DFF27EE0FFF1FEA59F84F06
:107BB000408151814A5B5F4F14F00C94A35591E0D2
:107BC0009093630688EE93E09093E0038093DF0345
:107BD00020919607E22FFF27EE0FFF1FEA59F84F7B
:107BE000808191818B5A9F4F0CF096CC2091970702
:107BF000E22FFF27EE0FFF1FEA59F84F60817181D6
:107C0000655B7F4F14F00C949E5230903C043320FF
:107C100011F00C949E528091D2048F5F893C10F435
:107C20000C94295578EC7093D20441E050E05093C5
:107C300019044093180451E050933C041092BB0483
:107C40001092BC041092BD041092BE041092610404
:107C500010926204109263041092640410925D0406
:107C600010925E0410925F041092600410927104EE
:107C700010927204109273041092740410926904AA
:107C800010926A0410926B0410926C04209091047C
:107C900030909204409093045090940420926D048C
:107CA00030926E0440926F04509270048090890468
:107CB00090908A04A0908B04B0908C04809265040C
:107CC00090926604A0926704B09268041092B30484
:107CD0001092B4041092B5041092B6041092B70436
:107CE0001092B8041092B9041092BA04909117043B
:107CF0009860909317045090C70751FC02C00C94F1
:107D0000A05270909C0770FE10C000911C0310914F
:107D10001D03075B134038F4A0911C03B0911D03B1
:107D2000AE5EB24010F40E9480140E947C2C209120
:107D300097070C94A05260926D0470926E0480922A
:107D40006F049092700453CA8093710490937204EC
:107D5000A0937304B093740417CA808191818358EF
:107D60009F4F861797070CF0EECA6115710509F44D
:107D7000EACACB010197E2CA4081518143585F4F63
:107D80004A175B070CF0C4CA109709F4C1CACD01A9
:107D90000197B9CA0081118103581F4F02171307B9
:107DA0000CF007CB2115310509F403CBC90101976C
:107DB000FBCA0081118103581F4F041715070CF0EF
:107DC000DDCA4115510509F4D9CACA010197D1CAC2
:107DD00029982CCB30909C0739AE7090320479866C
:107DE000772021F490913304992351F08091BA07C0
:107DF000992769817A818617970714F49A83898372
:107E00001885112311F40C940E4A1092400410921C
:107E10003F041092440410924304109242041092C2
:107E2000410480E090E0A8ECBFE38AAF9BAFACAF29
:107E3000BDAF80932A0890932B08A0932C08B09391
:107E40002D080F2EFBE06F2EFCEB7F2EF2E38F2E22
:107E5000FCE39F2EF02D22966CAE7DAE8EAE9FAED3
:107E600022976092150870921608809217089092D7
:107E700018081092320410923304198620910808D1
:107E80003091090840910A0850910B0880919104A3
:107E900090919204A0919304B09194048A8B9B8B4F
:107EA000AC8BBD8B280F391F4A1F5B1F80910F08B9
:107EB00090911008A0911108B0911208E0908904E7
:107EC000F0908A0400918B0410918C04EF8EF8A23C
:107ED00009A31AA38E0D9F1DA01FB11F8090FE073E
:107EE0009090FF07A0900008B09001088FA698AA74
:107EF000A9AABAAA60908D0470908E0480908F0415
:107F0000909090046E8A7F8A888E998E2FA438A8CC
:107F100049A85AA8260C371C481C591C2FA638AA59
:107F200049AA5AAAC090F307D090F407E090F50749
:107F3000F090F607CBA6DCA6EDA6FEA64090850441
:107F40005090860460908704709088044E865F8607
:107F5000688A798AABA4BCA4CDA4DEA4A40CB51C09
:107F6000C61CD71CABA6BCA6CDA6DEA6709133045A
:107F700023967FAF2397772309F0C5C459845520F2
:107F800009F0C1C480930F0890931008A0931108C2
:107F9000B0931208209308083093090840930A0808
:107FA00050930B0890909C08FFEF9F1609F413C59F
:107FB000E091A807AE2EBB24CC24DD246A897B89FE
:107FC0008C899D89A60195010E94696079018A01C9
:107FD0008091200890912108AA2797FDA095BA2F9B
:107FE000E81AF90A0A0B1B0B6F8D78A189A19AA1D7
:107FF000A60195010E94696059016A0180913308C8
:1080000090913408AA2797FDA095BA2FA81AB90A0B
:10801000CA0ADB0A292C332427FC3094432C532C26
:10802000C201B101A80197010E94F55F97FF02C04C
:108030000C94EE523B014C01A9E0959487947794FF
:108040006794AA95D1F7C201B101A60195010E94DA
:10805000F55F97FF02C00C94E8527B018C01F9E0B8
:1080600015950795F794E794FA95D1F7A0911C041C
:10807000B0911D04A134B10514F40C94EA4DD4015F
:10808000C30197FE02C00C944C543C014D019594E1
:10809000879477946794D801C70117FF02C00C94A6
:1080A00047547C018D0115950795F794E794D0907E
:1080B0009707ED2DFF27EE0FFF1FEA59F84F80813C
:1080C00091810190F081E02DF7FF02C00C94F452F1
:1080D0007A97A4F0C401B30123E030E040E050E01F
:1080E0000E94696039014A01C801B70123E030E00C
:1080F00040E050E00E94696079018A0180919E0809
:10810000282F332727FD3095432F532F261537056A
:108110004805590514F439014A01992787FD9095BE
:10812000909581959F4FAA2797FDA095BA2F681625
:1081300079068A069B0614F43C014D012E153F0575
:108140004007510714F479018A01E816F9060A0775
:108150001B0714F47C018D01A0907104B09072048F
:10816000C0907304D0907404A618B708C808D90842
:10817000A0927104B0927204C0927304D0927404FD
:108180004090690450906A0460906B0470906C0495
:108190004E185F08600A710A4092690450926A049E
:1081A00060926B0470926C040091EC031091ED03EB
:1081B0000F3F110509F010F40C94E7492396FFAC2A
:1081C0002397FF2029F49984992011F40C94634E8D
:1081D0002B961FAE1EAE2B974424552410925004AC
:1081E000A0900808B0900908C0900A08D0900B0829
:1081F00060900F08709010088090110890901208FD
:1082000020E030E040E050E022966CAD7DAD8EADD8
:108210009FAD22970E943D5F882311F00C94FA4C89
:1082200010923704109236041092350410923404E0
:10823000A092EE04B092EF04C092F004D092F10448
:108240006092F2047092F3048092F4049092F50428
:10825000109281041092820410928304109284047C
:1082600010927D0410927E0410927F04109280047C
:108270001092790410927A0410927B0410927C047C
:10828000109208081092090810920A0810920B0820
:1082900010920F08109210081092110810921208F4
:1082A0001092FE071092FF0710920008109201082A
:1082B0001092F3071092F4071092F5071092F60748
:1082C0001092ED031092EC03A0903F04B090400494
:1082D000C501B7FE02C00C94084A409764F088EECE
:1082E00093E090939B0380939A0359AC54FC03C092
:1082F00011E01093D704D090A507ED2CFF240027A0
:108300001127B501882777FD8095982F9501B7FE35
:1083100002C00C94384D442737FD4095542F0E94DD
:10832000F55F9B01AC01C801B7010E94F55F97FFA3
:1083300002C00C94324D39E09595879577956795F5
:108340003A95D1F76D2C77246A9C60016B9CD00C18
:108350007A9CD00C1124C601D7FE02C00C94084DA3
:108360009595879595958795680F791F2B016624BC
:1083700057FC6094762C4092BB045092BC046092EF
:10838000BD047092BE04209161043091620440915A
:1083900063045091640424193509460957092135AD
:1083A00003EC300700E0400700E0500714F40C94A1
:1083B000DD4920E533EC40E050E020936104309348
:1083C00062044093630450936404409161045091AB
:1083D00062046091630470916404405B5C436F4F7E
:1083E0007F4F64F400EB1CE32FEF3FEF0093610439
:1083F000109362042093630430936404E091570463
:10840000F0915804EF2B09F44EC1D9ACD3FE4BC107
:108410008A899B89AC89BD89B7FF02C00C949852A8
:1084200009E0B595A795979587950A95D1F72C0101
:1084300097FF02C00C9426538F8D98A1A9A1BAA1D1
:10844000B7FF02C00C94205319E0B595A7959795F6
:1084500087951A95D1F79C0197FF02C00C94305371
:10846000421653060CF42901B20157FE02C00C94C7
:108470002C534B0195948794959487949594879465
:108480000894811C911CA0915704B0915804A45EDB
:10849000BD4F7D010027F7FC0095102FA0902F08FD
:1084A000B0903008C0903108D0903208C601B501B4
:1084B0002BE035E040E050E00E946960E21AF30AE8
:1084C000040B150BC801B70128E631E040E050E08D
:1084D0000E946960DC01CB018C01045B104070904C
:1084E000D7047720A1F000E010E08091570490912C
:1084F0005804AA2797FDA095BA2FBC01CD012BE007
:1085000035E040E050E00E94F55F5B016C01E090D7
:108510009A03F0909B03E114F10491F439E14316BE
:10852000510474F460914E0470914F04600F711FF8
:1085300070934F0460934E04772011F00C946353B2
:10854000C801880F991F880F991F880F991FB401C0
:108550000E9434609B01442737FD4095542F2A0D1B
:108560003B1D4C1D5D1D20932F0830933008409318
:10857000310850933208D09089036D2D7727649D80
:10858000C001659D900D749D900D112497FF02C050
:108590000C943D53959587959595879595958795D9
:1085A00095958795959587958B01081B190B17FF56
:1085B00002C00C943553E114F10411F00C943E54B4
:1085C000E0901C04F0901D04A0901A04B0901B04CD
:1085D000EA0CFB1CF7FE02C00C94FB54F594E794E4
:1085E000F594E794F594E79480E490E0E80EF91EA2
:1085F000CA01B9012BE035E040E050E00E9469601B
:10860000DA01C9012091550430915604442737FD01
:108610004095542F821B930BA40BB50B845E9D4F8A
:10862000AF4FBF4FBC01CD0128E631E040E050E044
:108630000E946960DC01CB01845B9040809F400117
:10864000819F900C909F900C1124C401B7010E944F
:108650003460F3E0DF9E900111242617370714F4ED
:108660000C94405388279927821B930B681779072E
:108670000CF4BC016B01EE24D7FCE094FE2C60905E
:108680006104709062048090630490906404C60C4E
:10869000D71CE81CF91CC0926104D0926204E092DD
:1086A0006304F09264048091D60481508F3F09F4F2
:1086B000D1C68093D6042396FFAC2397FF2009F4FC
:1086C00018C68091F9079091FA07AA2797FDA095FF
:1086D000BA2FBC01CD010E94335FDC01CB012AAD72
:1086E0003BAD4CAD5DADBC01CD010E94AD5FDC0189
:1086F000CB01BC01CD010E94165FDC01CB01909340
:10870000FA078093F9079984992009F425C6809186
:10871000ED079091EE07AA2797FDA095BA2FBC010F
:10872000CD010E94335FDC01CB012AAD3BAD4CADE6
:108730005DADBC01CD010E94AD5FDC01CB01BC0190
:10874000CD010E94165FDC01CB019093EE07809370
:10875000ED078091250890912608AA2797FDA095FE
:10876000BA2FBC01CD010E94335F4B015C012AADE1
:108770003BAD4CAD5DADCA01B9010E948E5EDC011E
:10878000CB019C01AD01C501B4010E94AD5F1B018D
:108790002C018091750490917604A0917704B0919A
:1087A0007804BC01CD010E94335FDC01CB0122962D
:1087B0002CAD3DAD4EAD5FAD2297BC01CD010E9409
:1087C000AD5FDC01CB0120E030E040E05FE3BC01C5
:1087D000CD010E94AD5F9B01AC01C201B1010E94BD
:1087E0008E5EDC01CB01BC01CD010E94165FDC0175
:1087F000CB019093260880932508E090F907F0902C
:10880000FA07F0923507E09234070091ED071091D6
:10881000EE0710933707009336074091F907509100
:10882000FA074150504434F0A0E0B0E4B093FA07A6
:10883000A093F9076091F9077091FA076050704CA6
:1088400034F420E030EC3093FA072093F907E091FC
:10885000ED07F091EE07E150F04434F040E050E4D1
:108860005093EE074093ED070091ED071091EE074E
:108870000050104C34F480E090EC9093EE0780931D
:10888000ED07A0912508B0912608A150B04434F01E
:1088900060E070E470932608609325082091250815
:1088A000309126082050304C34F4E0E0F0ECF093A6
:1088B0002608E093250869807A80660C771C660C90
:1088C000771C39AC832D992780FF18C281FF4FC1D7
:1088D0008091D90799279C012071307084FD02C0D6
:1088E0000C94534E50918C0351555B3310F00C9403
:1088F000534E8091B70381508F3F11F40C94435332
:108900008093B7034FC11092810410928204109299
:1089100083041092840410927D0410927E041092BD
:108920007F04109280041092080810920908109297
:108930000A0810920B0810920F081092100810925B
:108940001108109212081FA618AA19AA1AAA20E044
:1089500030E040E050E02BA73CA74DA75EA7409138
:108960007104509172046091730470917404409387
:108970006D0450936E0460936F04709370040091C3
:10898000690410916A0420916B0430916C04009387
:108990006504109366042093670430936804109272
:1089A000ED031092EC0310923504109234041092EF
:1089B00037041092360423965FAD2397552309F0B0
:1089C000F3CBB985BB2309F0EFCB90909C08FFEF68
:1089D0009F1609F0EDCA3091A807E32EFF24002767
:1089E00011276A897B898C899D89A80197010E943A
:1089F000696039014A01C0902008D0902108160111
:108A0000442437FC4094542C6F8D78A189A19AA1FD
:108A1000A80197010E946960809133089091340801
:108A2000AA2797FDA095BA2F281B390B4A0B5B0B81
:108A3000621873088408950897FE02C00C946F545E
:108A400064E095948794779467946A95D1F757FF7B
:108A500002C00C94695479018A0144E01595079588
:108A6000F794E7944A95D1F740911C0450911D0466
:108A7000413451053CF420911A0430911B042134F7
:108A80003105A4F0C401B30123E030E040E050E040
:108A90000E94696039014A01C801B70123E030E052
:108AA00040E050E00E94696079018A01B090970728
:108AB000EB2DFF27EE0FFF1FEA59F84F80819181C0
:108AC0000190F081E02DF7FF02C00C9479547A9761
:108AD000A4F0C401B30123E030E040E050E00E9484
:108AE000696039014A01C801B70123E030E040E084
:108AF00050E00E94696079018A0191E2691671046F
:108B0000810491042CF030E2632E712C812C912C85
:108B1000A0EE6A16AFEF7A06AFEF8A06AFEF9A06BD
:108B200044F420EE622E2FEF722E2FEF822E2FEFC5
:108B3000922EB1E2EB16F104010511052CF090E242
:108B4000E92EF12C012D112DE0EEEE16EFEFFE06D1
:108B5000EFEF0E07EFEF1E070CF0FECA80EEE82ED7
:108B60008FEFF82E8FEF082F8FEF182FF5CA509048
:108B70008C03C0908003D0908103C50CD11C209140
:108B8000A1073327C29E2001C39E500CD29E500CD9
:108B90001124D2015497B0933904A0933804F1E022
:108BA000F093510440913A0450913B04D884DD2065
:108BB00021F0109239041092380420913804309139
:108BC0003904241735070CF099C0B0905104BB202C
:108BD00009F494C0421B530B80918B039927489F43
:108BE0007001499FF00C589FF00C1124C701F7FE4B
:108BF00002C00C947E549595879595958795930121
:108C0000281B390B8091EE039091EF0397FF02C070
:108C10000C94AA54959587958901081B190BC0904F
:108C20005904D0905A04E0905B04F0905C04F7FE85
:108C300002C00C94A05467E0F594E794D794C794CD
:108C40006A95D1F790918A03292F33274427552716
:108C5000C701B6010E94F55F97FF02C00C949A54B9
:108C600055E095958795779567955A95D1F731E0B9
:108C70006931730714F40C94045368E171E0061B26
:108C8000170B2090D4043090D50491012295329591
:108C9000307F3227207F322722193309200F311FDE
:108CA00037FF02C00C949654A901559547955595E8
:108CB00047955595479555954795BA01F0909D076D
:108CC0002F2D3327220F331F220F331F4217530735
:108CD00054F46216730614F0A901B9016216730602
:108CE00014F4A301B3016416750614F00C94FD523C
:108CF000A3017092D5046092D4043A0190902408A4
:108D00009C86892D9927880F991F880F991F805558
:108D10009040861597050CF43C01709219076092FB
:108D200018078091BB049091BC04A091BD04B09140
:108D3000BE04880F991FAA1FBB1F880F991FAA1F67
:108D4000BB1F8090250890902608881A990A61EA2E
:108D5000661671040CF4BBC2C30177FE02C00C940A
:108D6000DC5295958795881599050CF44C019095E2
:108D700081959F4F881699060CF44C01AC848A2D7E
:108D80009927880F991F880F991F9C012619370969
:108D9000281539050CF449019301281B390B82165B
:108DA00093060CF44901E091F907F091FA0740901D
:108DB000430450904404E419F509F0930608E09345
:108DC000050820E030E040E050E022966CAD7DAD3B
:108DD0008EAD9FAD22970E943D5F882309F462C249
:108DE0008091B3049091B404A091B504B091B604FD
:108DF000BC01CD010E94335F5B016C016A897B89F4
:108E00008C899D890E94335FDC01CB0122962CADB9
:108E10003DAD4EAD5FAD2297BC01CD010E94AD5F6F
:108E20007B018C01C201AA2797FDA095BA2FBC0136
:108E3000CD010E94335F9B01AC01C801B7010E94C4
:108E40008D5EDC01CB019C01AD01C601B5010E9424
:108E50008E5EDC01CB01BC01CD010E94165FDC01FE
:108E6000CB018093B3049093B404A093B504B09362
:108E7000B604A090B304B090B404C090B504D090F0
:108E8000B604F1E0AF16FAEFBF06F0E0CF06F0E06F
:108E9000DF0674F040E05AEF60E070E04093B30406
:108EA0005093B4046093B5047093B6045A016B01F7
:108EB00000E0A01606E0B0060FEFC0060FEFD006E8
:108EC00074F400E016E02FEF3FEF0093B30410932B
:108ED000B4042093B5043093B6045801690180911D
:108EE000050890910608AA2797FDA095BA2FBC0106
:108EF000CD010E94335F7B018C01C601B5010E9448
:108F0000335FDC01CB0120908E0330908F034090C3
:108F1000900350909103A2019101BC01CD010E94E8
:108F2000AD5F9B01AC01C801B7010E948E5EDC0100
:108F3000CB01BC01CD010E94165FDC01CB018C018D
:108F4000509182035E8F652F772788279927940198
:108F500097FC15C637FD00C635952795260D371D9C
:108F6000442737FD4095542F0E94F55F97FD02C6B8
:108F700026E095958795779567952A95D1F79B017A
:108F8000601771070CF48B0188279927821B930BBC
:108F9000081719070CF48C01C301800F911F880D6D
:108FA000991D97FD15C6959587959595879597FD7C
:108FB0000CC67C85272F3327281739070CF4C901E5
:108FC000B091FC07BD872B2F3327821793070CF432
:108FD000C9018093EF07C301801B910B880D991D78
:108FE00097FDF1C5959587959595879597FDE0C572
:108FF0001C85212F3327281739070CF4C901FD855B
:109000002F2F3327821793070CF4C9018093F80799
:10901000A091ED07B091EE07609141047091420478
:1090200029967FAF6EAF2997A61BB70BB093EC07BD
:10903000A093EB0720E030E040E050E022966CADDA
:109040007DAD8EAD9FAD22970E943D5F882309F4D0
:1090500014C18091B7049091B804A091B904B09163
:10906000BA04BC01CD010E94335F5B016C016F8DBE
:1090700078A189A19AA10E94335FDC01CB012296DD
:109080002CAD3DAD4EAD5FAD2297BC01CD010E9430
:10909000AD5F7B018C0129962EAD3FAD2997C901AB
:1090A000AA2797FDA095BA2FBC01CD010E94335F7E
:1090B000DC01CB019C01AD01C801B7010E948D5EAE
:1090C000DC01CB019C01AD01C601B5010E948E5EA1
:1090D000DC01CB01BC01CD010E94165FDC01CB019C
:1090E0008093B7049093B804A093B904B093BA04E2
:1090F000A090B704B090B804C090B904D090BA045E
:1091000031E0A3163AEFB30630E0C30630E0D306F1
:1091100074F040E05AEF60E070E04093B704509381
:10912000B8046093B9047093BA045A016B0140E02B
:10913000A41646E0B4064FEFC4064FEFD40674F40D
:1091400000E016E02FEF3FEF0093B7041093B80450
:109150002093B9043093BA04580169018091EB0758
:109160009091EC07AA2797FDA095BA2FBC01CD01DD
:109170000E94335F7B018C01C601B5010E94335F01
:10918000DC01CB01A2019101BC01CD010E94AD5FC8
:109190009B01AC01C801B7010E948E5EDC01CB01CE
:1091A000BC01CD010E94165FDC01CB018C013E8C1D
:1091B000632D772788279927940197FCFFC437FDF3
:1091C000FAC435952795260D371D442737FD409560
:1091D000542F0E94F55F97FDE6C4E6E095958795CC
:1091E00077956795EA95D1F79B01601771070CF4A5
:1091F0008B0188279927821B930B081719070CF4FA
:109200008C01C301800F911F8819990997FDC9C46A
:10921000959587959595879597FDC0C44C84242D89
:109220003327281739070CF4C9015D84252D33270E
:10923000821793070CF4C90180931C08C301801B9B
:10924000910B8819990997FD9FC4959587959595D8
:10925000879597FDA0C47C84272D332728173907CD
:109260000CF4C9016D84262D33278217930714F05F
:109270000C947B56C9010C947B568091EB0790911E
:10928000EC07AA2797FDA095BA2FC090B704D090FD
:10929000B804E090B904F090BA048C0D9D1DAE1D89
:1092A000BF1D1ECF8091050890910608AA2797FD43
:1092B000A095BA2FC090B304D090B404E090B50448
:1092C000F090B6048C0D9D1DAE1DBF1DCACD81E56D
:1092D000881691041CF070E5872E912C90EB89166E
:1092E0009FEF99060CF04ACD60EB862E6FEF962E1D
:1092F00045CD6A897B898C899D890E94335FDC0119
:10930000CB0122962CAD3DAD4EAD5FAD2297BC0199
:10931000CD010E94AD5F3B014C018091F907909116
:10932000FA07AA2797FDA095BA2FBC01CD010E948C
:10933000335FDC01CB012AAD3BAD4CAD5DADBC0173
:10934000CD010E94AD5FDC01CB019C01AD01C401E8
:10935000B3010E948E5ECBC96F8D78A189A19AA1BD
:109360000E94335FDC01CB0122962CAD3DAD4EADAA
:109370005FAD2297BC01CD010E94AD5F2B013C0186
:109380008091ED079091EE07AA2797FDA095BA2F3F
:10939000BC01CD010E94335FDC01CB012AAD3BADA6
:1093A0004CAD5DADBC01CD010E94AD5F9B01AC0138
:1093B000C301B2010E948E5EC0C920936104309344
:1093C000620440936304509364040C94E5418BA4BD
:1093D0009CA4ADA4BEA48092F3079092F407A0923F
:1093E000F507B092F607AFA4B8A8C9A8DAA8A0926A
:1093F000FE07B092FF07C0920008D0920108A0902B
:109400003F04B0904004C501B7FC02C00C946D410C
:10941000882799278A199B090C946D4180902A0806
:1094200090902B08A0902C08B0902D088AAE9BAE8F
:10943000ACAEBDAEE0901508F0901608009117088C
:10944000109118082296ECAEFDAE0EAF1FAF22971A
:109450000C943E3F98E19093D604B090A8072B2C33
:109460003324442455246A897B898C899D89A201EF
:1094700091010E94696030930B0720930A076F8D5A
:1094800078A189A19AA1A20191010E9469603093FB
:109490000D0720930C07A0912008B0912108B093EC
:1094A0000F07A0930E07E0903308F0903408F09275
:1094B0001107E092100700912508109126081093DB
:1094C00013070093120740903A0450903B045092C7
:1094D0001507409214078091590490915A04A09165
:1094E0005B04B0915C04B7FF02C00C940E5319E00A
:1094F000B595A795979587951A95D1F790931707E6
:1095000080931607809057049090580490921B0700
:1095100080921A07E0912203F0912303F0931D0734
:10952000E0931C0780912F0890913008A09131089A
:10953000B0913208BC01CD012BE035E040E050E0B5
:109540000E94696030932107209320078091450491
:10955000992790931F0780931E07A0909A08B090B8
:109560009B08B0922D07A0922C072091980830916B
:10957000990830932F0720932E078091630699272F
:1095800090933107809330076091DC037091DD0385
:1095900070933307609332078EC88091FF039091D8
:1095A0000004835F934034F0A8EEB3E0B093EE077D
:1095B000A093ED070091FF03109100040A5F134090
:1095C00014F40C9436380C943038409101045091C6
:1095D0000204435F534034F088EE93E09093FA071F
:1095E0008093F90760910104709102046A5F7340EF
:1095F00014F40C942F390C9429392B96AEADBFADD1
:109600002B97B0933E04A0933D04309240042092E7
:109610003F042BA83CA830924204209241044DA85C
:109620005EA8509244044092430440913D045091FE
:109630003E0457FD11C3B0919C07B9AFB2FF0CC0F7
:109640000F2EF0E0EF2EF0E0FF2EF0E00F2FF0E015
:109650001F2FF02D5701680120E030E040E050E07E
:10966000C401B3010E943D5F88230CF042C10F2E5C
:10967000F0E06F2EF0E07F2EF0E08F2EF0E09F2ED6
:10968000F02D60922A0870922B0880922C089092FC
:109690002D0820E030E040E050E0C601B5010E9416
:1096A0003D5F88230CF038C10F2EF0E0EF2EF0E084
:1096B000FF2EF0E00F2FF0E01F2FF02DE0921508A5
:1096C000F09216080093170810931808409143046D
:1096D00050914404CA0157FD2EC1959587959595E3
:1096E000879597FD2FC120911C0430911D042817E8
:1096F00039070CF032C1CA0157FD98C797FD94C7CE
:10970000BC017595679575956795653671050CF47F
:1097100027C164E670E04091410450914204CA01BF
:1097200057FF25C10396959587959595879597FF42
:1097300024C1909581959F4F20911A0430911B046C
:10974000281739070CF421C1C9010197F09152047F
:10975000F887FF2309F42EC110921D0410921C04F7
:1097600010921B0410921A04F8ACAF2DBB27AA0F5D
:10977000BB1FAA59B84F4091BB07842E99240D9165
:109780001C918016910624F4D090D907D2FC42C2D5
:10979000B8ACEB2DFF27EE0FFF1FEA59F84FC42E90
:1097A000DD249090BC07C918D108A080B180AC140A
:1097B000BD0414F41092310438ACA32DBB27AA0FBA
:1097C000BB1FAA59B84F242F332744245524421ACB
:1097D000530A2D903C902414350424F47090D9073A
:1097E00073FC14C210913004112391F058ADE52F91
:1097F000FF27EE0FFF1FEA59F84F8091BC0799270A
:10980000841B910960817181861797070CF47FC6CC
:109810007FA9A72FBB27AA0FBB1FAA59B84F642E39
:1098200077248D919C916816790624F45090D9077D
:1098300050FCE7C150912E04552399F00FA9A02F99
:10984000BB27AA0FBB1FAA59B84FE42EFF24F091E3
:10985000BC07EF1AF1088D909C908E149F040CF4B5
:1098600052C6FFA8EF2DFF27EE0FFF1FEA59F84F52
:10987000442E5524CC24DD24C418D508A080B18002
:10988000AC14BD0424F4D090D907D1FCB6C13091FA
:109890002F04332391F09FA8A92DBB27AA0FBB1F2C
:1098A000AA59B84F8091BC079927841B91092D9024
:1098B0003C90821593050CF423C6B0903104BB2074
:1098C00029F480913004882309F495C191E055234F
:1098D00029F480912F04882309F487C121E0209383
:1098E00033041092320410923104109230040C941C
:1098F000ED3E60922A0870922B0880922C0890927C
:109900002D0820E030E040E050E0C601B5010E94A3
:109910003D5F88230CF4C8CEE0921508F09216083B
:109920000093170810931808409143045091440481
:10993000CA0157FFD2CE0396959587959595879541
:1099400097FFD1CE909581959F4F20911C04309127
:109950001D04281739070CF4CECEB90161507040B0
:109960004091410450914204CA0157FDDBCE9595C8
:1099700087959595879597FDDCCE20911A043091B7
:109980001B04281739070CF0DFCECA0157FD52C659
:1099900097FD54C69595879595958795853691053C
:1099A0000CF4D4CE84E690E0F0915204F887FF23C3
:1099B00009F0D2CE90931B0480931A0470931D0477
:1099C00060931C04D1CE10923C04109252041B856B
:1099D0001A3011F00C94493A289AE0911804F09149
:1099E0001904E95EF34010F00C94573A10923C04CD
:1099F0000C948C3A50923704409236042B964EAD1C
:109A00005FAD2B9750933504409334040C94184168
:109A100003960C94B041F8E74F2FF7E15F2FF7E082
:109A20006F2F712DE40EF51E061F171F0C946D3657
:109A30002F5F3F4F4F4F5F4F0C9472350894E11CDE
:109A4000F11C011D111D0C9451350894E11CF11CF1
:109A5000011D111D0C94263521503E4F4F4F5F4F75
:109A60000C945A3861507E4F8F4F9F4F0C949B41FE
:109A7000222733272A193B090C948B4110924B045F
:109A800010924A0457FD02C00C94F939109249040F
:109A90001092480437FD02C00C94073A1092470414
:109AA000109246040C94113A10924D0410924C04FA
:109AB0000C94E73921503E4F4F4F5F4F0C946E3757
:109AC0001F81112311F00C946D39B0913204BB2326
:109AD00011F00C946D390091F9071091FA07093CC7
:109AE00011050CF0ACC68091F9079091FA078853E4
:109AF0009F4FA4F48091F9079091FA07880F991F5E
:109B0000880F991FC090F907D090FA078C0D9D1D02
:109B1000805E9C4F9093FA078093F9076091ED0760
:109B20007091EE07693C71050CF423C78091ED0735
:109B30009091EE07880F991F880F991F4090ED07AD
:109B40005090EE07840D951D805293409093EE0740
:109B50008093ED070C946D392F5F3F4F3595279516
:109B6000260D371D442737FD4095542F0E94F55F81
:109B700097FFFEC9615C7F4F8F4F9F4FF9C9222726
:109B8000332728193909E6C9039695958795959540
:109B9000879597FF60CB80E090E064CB80E090E019
:109BA00044CB039635CB615C7F4F8F4F9F4F15CBD6
:109BB00080E090E024CA2F5F3F4F03CB222733275A
:109BC00028193909FCCA03960DCA80E090E0F8C94B
:109BD0000396E9C960911A0470911B046134710500
:109BE00014F40C9457400C943F40909332048093AB
:109BF00033040C94ED3E982F6ACE41E040932F043D
:109C00005CCEB1E0B0932E045B2F2BCE91E090930D
:109C10003004FECD31E030933104CECD2B96EEAD45
:109C2000FFAD2B97F0933E04E0933D043092400447
:109C300020923F046BA97CA9709342046093410475
:109C40002DA93EA9309344042093430440913D0440
:109C500050913E0457FFEFCC10923E0410923D0409
:109C6000EACC3DE7E32EF12C012D112DAEE76A166B
:109C700071048104910414F00C94223BB3E86B1638
:109C8000BFEF7B06BFEF8B06BFEF9B0614F00C9473
:109C9000273B83E8682E8FEF782E8FEF882E8FEF8B
:109CA000982E0C94273B232B31F470918C03723344
:109CB00010F40C94794411E01093510488EC8093D3
:109CC000B7030C94D24530905004332011F00C941B
:109CD000E8408FA498A8A9A8BAA88092FE079092FD
:109CE000FF07A0920008B09201086BA47CA48DA489
:109CF0009EA46092F3077092F4078092F507909209
:109D0000F6078091080890910908A0910A08B0917F
:109D10000B08B7FDA5C5292E3A2E4B2E552447FC1E
:109D20005A94209208083092090840920A085092EA
:109D30000B0880910F0890911008A0911108B09124
:109D40001208B7FDC5C6C92EDA2EEB2EFF24E7FC9C
:109D5000FA94CB82DC82ED82FE82C0920F08D09210
:109D60001008E0921108F09212087090A807E72CF2
:109D7000FF24002711272091810430918204409113
:109D8000830450918404C801B7010E94F55F97FDD8
:109D90009AC6672E782E892E992487FC9A94209152
:109DA0007D0430917E0440917F0450918004C8016D
:109DB000B7010E94F55F97FD95C6E72EF82E092F93
:109DC000112707FD1A95D201C10186199709A80923
:109DD000B9097091C107272E332444245524BC01AE
:109DE000CD01A20191010E9469602BA33CA34DA368
:109DF0005EA32FA338A749A75AA78B819C81AD8169
:109E0000BE818E199F09A00BB10BBC01CD01A2012F
:109E100091010E9469608BA19CA1ADA1BEA1B7FD7B
:109E20005CC6892F9A2FAB2FBB27A7FDBA952B961F
:109E30009FAF8EAF2B9757FD41C6BB2757FDBA95F5
:109E4000A52F942F832F2C01A0911C04B0911D04E9
:109E5000A134B105C4F460911A0470911B046134FB
:109E600071058CF490919707E92FFF27EE0FFF1FE4
:109E7000EA59F84F808191810190F081E02DF7FD42
:109E8000C6C67A972CF010919C081F3F09F4B9C5FB
:109E90004E895F89688D798D0A891B892C893D8956
:109EA000401B510B620B730B4093BF045093C004D3
:109EB0006093C1047093C204EE84FF8408891989F9
:109EC0006F8C78A089A09AA0E618F70808091909EC
:109ED000E092C304F092C4040093C5041093C60436
:109EE0004093C7045093C8046093C9047093CA0494
:109EF000E092CB04F092CC040093CD041093CE04F6
:109F0000A0906D04B0906E04C0906F04D090700467
:109F1000A41AB50AC60AD70AA0926D04B0926E04BC
:109F2000C0926F04D0927004809165049091660491
:109F3000A0916704B09168048E199F09A00BB10B22
:109F40008093650490936604A0936704B0936804BB
:109F500020914E0430914F042138310594F0E09166
:109F6000A504F091A6043196F093A604E093A5040D
:109F7000A0911308B09114081196B0931408A093FF
:109F8000130820583F4F94F4A091A504B091A60463
:109F90001197B093A604A093A50480911308909103
:109FA00014080197909314088093130860900F0889
:109FB00070901008809011089090120810924F0431
:109FC00010924E0421E030E08091EE049091EF0475
:109FD000A091F004B091F104A0900808B090090895
:109FE000C0900A08D0900B088A199B09AC09BD09DA
:109FF000815E914BAF4FBF4F8F539C49A040B04003
:10A0000008F464C430909D08B0E3B3150CF024C587
:10A01000413080E1580780E0680780E078070CF461
:10A02000E3C4F091EA04FF2309F481C52B962EAD19
:10A030003FAD2B973093350420933404DB01CA01E4
:10A0400077FD3AC6B7FD44C62CE0B595A795979520
:10A0500087952A95D1F701969093E9048093E804B7
:10A06000DB01CA0177FD30C6F3E0B595A79597955A
:10A070008795FA95D1F78FA398A7A9A7BAA7619654
:10A080008CAF9DAFAEAFBFAF619789589341A040F1
:10A09000B04074F088E893E1A0E0B0E08FA398A707
:10A0A000A9A7BAA761968CAF9DAFAEAFBFAF6197BE
:10A0B00061968CAD9DADAEADBFAD6197B7FDD7C517
:10A0C000892F9A2FAB2FBB27A7FDBA952B96EEAD04
:10A0D000FFAD2B97E80FF91F2B96FFAFEEAF2B9735
:10A0E0004030F0EF5F07FFEF6F07FFEF7F070CF0E7
:10A0F00069C42090EB04222009F4F9C42B96AEAD7C
:10A10000BFAD2B97B0933504A0933404DB01CA0193
:10A1100077FD8DC527968CAF9DAFAEAFBFAF2797AC
:10A12000B7FD91C527968CAD9DADAEADBFAD279760
:10A130003CE0B595A795979587953A95D1F72796E1
:10A140008CAF9DAFAEAFBFAF27972091E8043091A1
:10A15000E90425968EAD9FAD2597280F391F3093C2
:10A16000E9042093E804DB01CA0177FD68C523E018
:10A17000B595A795979587952A95D1F78837ECEEF1
:10A180009E07EFEFAE07EFEFBE0724F488E79CEEE3
:10A19000AFEFBFEF8093D8049093D904A093DA0473
:10A1A000B093DB04B7FD7BC5892F9A2FAB2FBB275C
:10A1B000A7FDBA95E0913404F0913504E80FF91F3A
:10A1C0002B96FFAFEEAF2B97F091C2078F2F9927F9
:10A1D0002091E8043091E904821793072CF49093BE
:10A1E000E9048093E8049C0122953295307F322760
:10A1F000207F3227A32DBB27A7FDB095A217B30759
:10A2000074F4832D37FCFAC48595859585958595DD
:10A21000992787FD90959093E9048093E804413055
:10A2200094E0590790E0690790E0790774F0809115
:10A23000A9049091AA042091E8043091E904820FC6
:10A24000931F9093AA048093A90440505C4F6F4FD2
:10A250007F4F74F46091A9047091AA044091E804BE
:10A260005091E904641B750B7093AA046093A904D0
:10A2700021E030E08091F2049091F304A091F40485
:10A28000B091F50486199709A809B909815E914B27
:10A29000AF4FBF4F8F539C49A040B04020F050E3D8
:10A2A00053150CF0F0C351E0E51650E1F50650E00F
:10A2B000050750E015070CF476C37091EC04772382
:10A2C00009F425C45092370440923604D801C701DE
:10A2D00017FDEAC4B7FDC6C43CE0B595A7959795B0
:10A2E00087953A95D1F701969093E9048093E80415
:10A2F000D801C70117FDB2C423E0B595A79597957E
:10A3000087952A95D1F7893863E1960760E0A6071B
:10A3100060E0B60724F088E893E1A0E0B0E0809325
:10A32000DC049093DD04A093DE04B093DF048091FD
:10A33000DC049091DD04A091DE04B091DF04B7FD50
:10A340009BC4892F9A2FAB2FBB27A7FDBA954090AE
:10A35000360450903704480E591E80E0E81680EF0E
:10A36000F8068FEF08078FEF18070CF03AC330910B
:10A37000ED04332309F4E3C35092370440923604CA
:10A38000D801C70117FD4BC49C01AD01B7FD82C4C4
:10A390007CE055954795379527957A95D1F740906C
:10A3A000E8045090E904420E531E5092E904409292
:10A3B000E804D801C70117FD69C463E0B595A79506
:10A3C000979587956A95D1F78837ECEE9E07EFEF62
:10A3D000AE07EFEFBE0724F488E79CEEAFEFBFEFC8
:10A3E0008093DC049093DD04A093DE04B093DF043B
:10A3F0008091DC049091DD04A091DE04B091DF0433
:10A40000B7FD3FC4892F9A2FAB2FBB27A7FDBA9565
:10A410004090360450903704480E591E8F2F9927CC
:10A420002091E8043091E904821793072CF490936B
:10A43000E9048093E8049C0122953295307F32270D
:10A44000207F3227632D772767FD7095621773078A
:10A4500074F4832D37FCD0C38595859585958595B6
:10A46000992787FD90959093E9048093E804F1E0A3
:10A47000EF16F4E0FF06F0E00F07F0E01F0774F0BE
:10A480002090A7043090A8042091E8043091E904BA
:10A49000220E331E3092A8042092A70420E0E21678
:10A4A0002CEFF2062FEF02072FEF120714F00C9497
:10A4B0000041E090A704F090A8040091E8041091F6
:10A4C000E904E01AF10AF092A804E092A7040C94BF
:10A4D0000041B0913C04BB2311F40C94D33C809117
:10A4E000180490911904FFEF8F3F9F0711F40C940B
:10A4F000D73C019690931904809318040C94D73C90
:10A5000010922F04DAC910922E0450E0AAC91092BA
:10A5100030047EC908E91AE31093E0030093DF03D7
:10A5200080E09CE090931203809311030C94373ADF
:10A5300081509E4FAF4FBF4F0C9410421092D204E7
:10A54000E22FFF27EE0FFF1FEA59F84F20813181DC
:10A550002C3431050CF44DC08091D3048F5F893CBD
:10A5600008F4ADC010923C0418EC1093D304109280
:10A570001904109218040C948C3A3091170432602C
:10A58000309317040C94F23C20E030E040E853E4B0
:10A590000E948E5E0C94053C2D5F3F4F0C94BE3B99
:10A5A0002D5F3F4F0C948B3B20E030E040E853E4BC
:10A5B0000E948E5E0C94273C01960C94B1462B961B
:10A5C0008EAD9FAD2B9790933E0480933D042DC894
:10A5D00061507E4F8F4F9F4F0C942D4061507E4FA6
:10A5E0008F4F9F4F0C941A40F095E195FF4F0C94BC
:10A5F00068401092D3040C948C3A7093D504609305
:10A60000D4043A010C947E464EEF683E740714F071
:10A610000C943F4668EE7EEF0C943F4681509E4F6F
:10A62000AF4FBF4F0C94774A03966AC890958195B7
:10A630009F4F64C8909581959F4FAAC90396AAC958
:10A6400081509E4FAF4FBF4F0C9424425094419481
:10A65000510853940C941C42695F7F4F0C9439420B
:10A66000309521953F4F0C94304244EF51E0509388
:10A670009B0340939A030C9453434F960C94CA4205
:10A68000B9010C943A4340911C0350911D03495E5B
:10A69000534008F4D2C19091F0039A509093F00384
:10A6A000B0915907B91BB7BD8CE291E09093E003DC
:10A6B0008093DF038AEF8093B7030C94D245809395
:10A6C000D3040C948C3A28EC30E03093E0032093D0
:10A6D000DF03C601B5012BE035E040E050E00E9409
:10A6E000696030935604209355041092D7040C945B
:10A6F000A04240815181455B5F4F0CF0DBC110915E
:10A70000D1041F5F1093D104193C10F40C94EA3D5E
:10A71000BB85BC3008F074C2299874E0E72E70E065
:10A72000F72EFFEFD7010F2E0E94916010923C048C
:10A730001092D10410921904109218040E947C2CDB
:10A7400080919F049091A00497FDD2C2892F990F08
:10A75000990BD701082E0E949160D7011196809124
:10A760009F049091A004082E0E949160D701129638
:10A7700080919D0490919E0497FDB7C2892F990FF7
:10A78000990B082E0E949160D701139680919D0429
:10A7900090919E04082E0E94916087010C5F1F4FCC
:10A7A0008091970490919804A0919904B0919A0493
:10A7B000BC01CD010E94165FDC01CB019C0197FD1D
:10A7C00091C2832F992787FD9A95D801082E0E9460
:10A7D000916087010B5F1F4F8091970490919804BF
:10A7E000A0919904B0919A04BC01CD010E94165F1A
:10A7F000DC01CB01D801082E0E9491600E94200349
:10A80000F82EFA943FEFF31611F40C94E83D04E6A9
:10A8100010E0B0903C04BB2011F00C94E83D109384
:10A82000E0030093DF038AEF90E00E940F13FA9495
:10A830002FEFF21671F7209196070C94EA3D809164
:10A84000F9079091FA07880F991F880F991FA09018
:10A85000F907B090FA078A0D9B1D805293405AC9A0
:10A8600081509F4FAF4FBF4F56CA909580957095BE
:10A8700061957F4F8F4F9F4F0C9418370894E108D4
:10A88000F108F0929B03E0929A030C9453430196D3
:10A89000A11DB11D0C9451400196A11DB11D0C9438
:10A8A0004540F1E0F093D7041092BB041092BC0431
:10A8B0001092BD041092BE041092610410926204C2
:10A8C00010926304109264040C94F23C30909D0842
:10A8D0009FCB215F3F4F4F4F5F4F0C942B458FE035
:10A8E00090E0A0E0B0E0680E791E8A1E9B1E0C94DA
:10A8F0002045F095E195FF4F0C94674503960C9425
:10A90000FB4590958095709561957F4F8F4F9F4F38
:10A910000C940D376150704F8F4F9F4F0C94BA3687
:10A920002150384F4F4F5F4F0C94A536215F3F4F5A
:10A930000C945446615E7F4F8F4F9F4F0C9430466E
:10A940006FE770E080E090E0C60ED71EE81EF91EAB
:10A950000C941B4601960C940A466150704F8F4F21
:10A960009F4F0C94F6362150384F4F4F5F4F0C9449
:10A97000E736A091ED07B091EE07A853BF4F14F052
:10A980000C946D398091ED079091EE07880F991F17
:10A99000880F991FE090ED07F090EE078E0D9F1D38
:10A9A000805E9C4FD3C81092DC041092DD0410929C
:10A9B000DE041092DF043093E9042093E80410923F
:10A9C000EC04CBCC8FA198A5A9A5BAA58093D804F7
:10A9D0009093D904A093DA04B093DB041092EB04B3
:10A9E000F3CB1092ED041ACD3093E9042093E804E0
:10A9F0001092EA0475CBE7E0F0E0EE0EFF1E0C9437
:10AA0000EE422B964EAD5FAD2B975093350440939D
:10AA100034045092370440923604CA0157FDFDC0F9
:10AA2000959587952B969FAF8EAF2B97C20157FCBC
:10AA3000F2C02C01559447942BCA00911C0310912D
:10AA40001D030436110508F0BDC09091F003965F18
:10AA500025CE8093D20474CD8BA19CA1ADA1BEA1C3
:10AA60008093D8049093D904A093DA04B093DB04C4
:10AA70001092E9041092E804A8EEB3E0B0939B03AF
:10AA8000A0939A03A1CB1092DC041092DD041092E3
:10AA9000DE041092DF041092E9041092E804A8EE9C
:10AAA000B3E0B0939B03A0939A03B8CC8093D104F6
:10AAB0000C94EA3D3093D1040C94EA3D21503F4F71
:10AAC0004F4F5F4FBAC961507F4F8F4F9F4F61C942
:10AAD00081509F4FAF4FBF4F36C981509F4FAF4FEF
:10AAE000BF4F9FC961507F4F8F4F9F4F66C98FA146
:10AAF00098A5A9A5BAA58093D8049093D904A0934A
:10AB0000DA04B093DB0491E09093EB045DCB1092F8
:10AB1000DC041092DD041092DE041092DF04309306
:10AB2000E9042093E804B1E0B093EC0416CC309330
:10AB3000E9042093E80431E03093EA04D1CAE1E06B
:10AB4000E093ED046BCC0E94200346E564E977E0D6
:10AB50000E94C90240909C0740FE0EC060911C03F9
:10AB600070911D03675B734050F500911C031091B9
:10AB70001D030E5E124018F10E947C2C0E942003DF
:10AB8000F82EFA945FEFF51611F40C94E83D04E604
:10AB900010E0E0903C04EE2011F00C94E83D10939E
:10ABA000E0030093DF038AEF90E00E940F13FA9412
:10ABB0007FEFF71671F7209196070C94EA3D0E94FB
:10ABC0008014DACF40913A0450913B0444515040F4
:10ABD00050933904409338044C5E5F4F10925104F7
:10ABE00031E03093B7030C94D645299A0C94213D5B
:10ABF000209195070C944D3D815F2ECC815F04CB55
:10AC0000299A8BCDF095E195FF4F0C94CC3DF095B2
:10AC1000E195FF4F36C901960CCF019601CF8827E9
:10AC20009927DC018E199F09A00BB10BADCB8827AA
:10AC30009927DC01841B950BA60BB70B6BCA0796F3
:10AC4000A11DB11D94CA8150904FAF4FBF4F2796A1
:10AC50008CAF9DAFAEAFBFAF279764CA0796A11D5B
:10AC6000B11D4ACB8150904FAF4FBF4F35CB815074
:10AC70009F4FAF4FBF4F24CA81509F4FAF4FBF4F21
:10AC800060CB81509F4FAF4FBF4FBCCB0796A11DEC
:10AC9000B11D93CB2150304F4F4F5F4F79CB815037
:10ACA0009F4FAF4FBF4F80CA88279927DC018E196D
:10ACB0009F09A00BB10B0ECB88279927DC01841BC1
:10ACC000950BA60BB70BBEC90796A11DB11DCCC92C
:10ACD0008150904FAF4FBF4FB7C9F095E195FF4FEF
:10ACE0000C94493D21503F4F6CCD81509F4F46CD34
:10ACF00081509F4F2BCD80931908C05BDF4F0FB65B
:10AD0000F894DEBF0FBECDBFDF91CF911F910F91A1
:10AD1000FF90EF90DF90CF90BF90AF909F908F907B
:10AD20007F906F905F904F903F902F90089520916B
:10AD300002053091030540910405509105052093CB
:10AD4000FA043093FB044093FC045093FD0480917B
:10AD5000FE049091FF04A0910005B091010580933D
:10AD6000F6049093F704A093F804B093F9040895BF
:10AD700010920D0510920C0510920B0510920A0509
:10AD8000089574B1706A74B93D9A62E56CBD1DBCDA
:10AD9000459A51E0509339084AEA40933D0833E818
:10ADA00030933E089AE090933F0810924108109229
:10ADB0004008109243081092420810925F081092C7
:10ADC000600827E4209361089093620883E08093F1
:10ADD00063080895F8948091910490919204A09151
:10ADE0009304B0919404BC01CD012CE630E040E026
:10ADF00050E00E94696030934108209340088091A0
:10AE0000890490918A04A0918B04B0918C04BC01B8
:10AE1000CD012CE630E040E050E00E9469603093C4
:10AE200043082093420880912F0890913008A09108
:10AE30003108B0913208BC01CD012BE035E040E093
:10AE400050E00E9469603093490820934808E091DF
:10AE50009B04F0919C0480910C0890910D08BF0117
:10AE60000E9434602CE030E0629FA001639F500D8F
:10AE7000729F500D112450934508409344088091CF
:10AE8000280890912908BF010E943460629FA001A8
:10AE9000639F500D729F500D1124509347084093AB
:10AEA000460810929C0410929B0410920D08109278
:10AEB0000C08109229081092280880913F089927C1
:10AEC0008217930709F489C0281739070CF46DC05D
:10AED0008A30910509F423C10B9709F4ABC078942B
:10AEE000E0915F08EE2309F48FC02091650830914E
:10AEF0006608B90161507E4F6F5F7340B0F44091B6
:10AF0000670850916808CA0181509E4F8F5F934037
:10AF100060F470919C0775FF08C030930D05209375
:10AF20000C0550930B0540930A0580916B08909196
:10AF30006C0821E08936920724F49093580480939A
:10AF400057048091570490915804209155043091F2
:10AF50005604821B930B845E9D4F68E671E00E944D
:10AF60003460845B90409093540480935304209108
:10AF70006F08309170084091DF035091E003421751
:10AF8000530740F450916306552321F43093E003B6
:10AF90002093DF038091640899278436910509F492
:10AFA000AEC087369105C9F108958D30910509F439
:10AFB000EFC00E9709F093CFA0916008A0935008BE
:10AFC0008091610880935108409162084093520833
:10AFD000F0916308F093530882CF80916306863026
:10AFE00018F01092630685E08093500860913A044F
:10AFF00070913B0470935308609352087894E091E9
:10B000005F08EE2309F071CF10920D0510920C0528
:10B0100010920B0510920A050895B0917108B09333
:10B020009C089091720890939E0830917308309319
:10B030009D08089540919607E42FFF27EE0FFF1F0C
:10B04000EA59F84F0190F081E02DE038F1050CF05D
:10B05000D0C05FEFE138F50714F4E1E8FFEFE093CB
:10B06000500880919707E82FFF27EE0FFF1FEA593E
:10B07000F84F0190F081E02DE038F1050CF4CCC0E0
:10B08000EFE7F0E0E0935108A0919507EA2FFF2742
:10B09000EE0FFF1FEA59F84F0190F081E02DE038E4
:10B0A000F1050CF4B1C0EFE7F0E0E0935208209115
:10B0B0009407E22FFF27EE0FFF1FEA59F84F019088
:10B0C000F081E02DE038F1050CF496C0EFE7F0E0F8
:10B0D000E0935308B0914C04B093540890914A0403
:10B0E0009093550870914804709356085091460407
:10B0F000509357083091450430935808F0CE809112
:10B10000710899279093990880939808A0917308E3
:10B11000B0917408B0939B08A0939A080895409149
:10B120002D044093500860912C0460935108E091E5
:10B130002B04E0935208F0912A04F0935308B09145
:10B140002904B09354089091280490935508709165
:10B150002704709356085091260450935708309155
:10B16000170430935808337F3093170480912203DB
:10B1700090912303809359082091AC0720935A089B
:10B18000A2E0B0E00E948460802D80935B08A7CE8F
:10B190006091CC0760935008E091CD07E09351088F
:10B1A000F091CE07F0935208B091CF07B0935308B7
:10B1B0009091D007909354087091D10770935508DF
:10B1C0005091D207509356083091D30730935708C7
:10B1D0002091D60720935808A091D407A09359082E
:10B1E0008091D50780935A088091D70780935B0898
:10B1F00076CEEFE7F0E033CF2FEFE138F2070CF037
:10B2000067CFE1E8FFEF64CF8FEFE138F8070CF08C
:10B210004CCFE1E8FFEF49CF6FEFE138F6070CF0D4
:10B2200031CFE1E8FFEF2ECF80913908882309F470
:10B230003BC045984DE358E050933B0840933A0893
:10B2400030910E05E32FFF27E854FC4F932F9F5FAB
:10B25000208120933F08963008F027C090930E0578
:10B26000109239080E94EA5661E060933C080000A1
:10B2700000000000000000000000000000000000CE
:10B2800000000000000000000000000000000000BE
:10B2900000000000000000000000000000005091CD
:10B2A0003D0850935C085EBD089510920E05D8CFFE
:10B2B00020913908222309F045C00DB407FE42C091
:10B2C00084E08093DE03459A3EB580910F0599276F
:10B2D0008130910509F437C0823091050CF451C0DA
:10B2E000029709F439C020913C08203208F030C0A0
:10B2F0004598000000000000000000000000000071
:10B30000000000000000000000000000000000003D
:10B31000000000000000000000000000000000002D
:10B320000000E0913A08F0913B08E20FF11D8081A6
:10B330008EBDB0915C089081B90FB0935C082F5F0F
:10B3400020933C080895353551F120930F05CBCF5C
:10B35000F1E0F0933908F3CF40915E08E42FFF2726
:10B36000E258F74F30834F5F40935E084A3100F157
:10B3700050911005351711F110925F0810920F05CA
:10B38000B2CF892B09F0AFCF20935E083093100520
:10B39000313809F0A8CF81E080930F05A4CF209128
:10B3A0001005230F2093100582E080930F059BCF9B
:10B3B00070911005730F7093100595CF6AE1EEE759
:10B3C000F8E0A4E6B8E001900D926A95E1F731E06B
:10B3D00030935F0810920F0586CF20E030E088237D
:10B3E00021F0809111058823B1F48091C607992737
:10B3F0008870907095958795959587959595879583
:10B4000028173907C1F0429A24E630E030933B0711
:10B4100020933A07089521E030E08091C6079927EC
:10B420008870907095958795959587959595879552
:10B430002817390741F7429810923B0710923A07B4
:10B44000089520E030E0882321F0809111058823C1
:10B45000C1F48091C6079927807190709595879562
:10B46000959587959595879595958795281739078B
:10B4700059F0439A24E630E030933D0720933C078F
:10B48000089521E030E0E5CF439810923D071092F7
:10B490003C07089587B18C6087B91092120510920D
:10B4A00011052091C60723FF11C0429A44E650E0DF
:10B4B00050933B0740933A0724FF0FC0439A24E67A
:10B4C00030E030933D0720933C070CC04298109227
:10B4D0003B0710923A0724FDF1CF439810923D07A5
:10B4E00010923C071092180530E83093BF03109279
:10B4F00015053093BE030895CF93809119058150AF
:10B500008F3F09F492C080931905C091C60720911E
:10B5100016054091130550E0222399F080911905FA
:10B5200070911705871708F45FC09091AC07292F19
:10B530003327A0912203B0912303A217B3070CF481
:10B5400053C020E030E0552329F0B0911105BB2312
:10B5500009F04CC0EC2FFF27E870F070F595E795E7
:10B56000F595E795F595E7952E173F0709F44EC039
:10B57000429A64E670E070933B0760933A0750E0AC
:10B58000442389F040911905F09114054F1750F1AB
:10B590003091AC07A32FBB27809122039091230306
:10B5A0008A179B07FCF020E030E0552321F05091F2
:10B5B0001105552389F5EC2FFF27E071F070F59503
:10B5C000E795F595E795F595E795F595E7952E17A8
:10B5D0003F0729F1439A24E630E030933D0720935A
:10B5E0003C071FC151E0DFCF51E0ABCF21E030E09D
:10B5F000EC2FFF27E870F070F595E795F595E79546
:10B60000F595E7952E173F0709F0B2CF42981092B3
:10B610003B0710923A07B3CF21E030E0CCCF4398FC
:10B6200010923D0710923C07FCC089E080931905F9
:10B63000C091C6078C2F992785FD30C086FFC1C0F9
:10B6400020913C04222371F530919607E32FFF27C8
:10B65000EE0FFF1FEA59F84F408151814C5A5F4F5E
:10B660000CF16081718165357105E4F450919707A3
:10B67000E52FFF27EE0FFF1FEA59F84FA081B18198
:10B68000A55BBF4F1CF471E070931205808191811E
:10B690008C3491053CF02093120504C080913C0449
:10B6A00080931205E09112054C2F5527BA01637063
:10B6B000707061157105C9F09091AC07292F33277F
:10B6C000A0912203B0912303A217B30774F442FDA3
:10B6D0007AC0E0931105809119056F5F7F4F99271C
:10B6E0000E9434606093190502C0E09311059091A7
:10B6F000C9079B3F08F43EC0E0910E08E73ED0F139
:10B700009091C807292F2078209316058091BF03B8
:10B71000892329F08091040867E10E9414608093D6
:10B7200017059091CB079B3FB0F030912308373E2F
:10B7300090F09091CA07492F40784093130580916B
:10B74000BE03892329F08091070867E10E941460F5
:10B7500080931405E0CE9B3FE0F0609123086A30AF
:10B76000C0F480E09091CA0797FF81E0482F409392
:10B770001305E5CF9B3FC8F0F0910E08FA30A8F40E
:10B7800080E09091C80797FF81E0282F209316054D
:10B79000BDCF8091150581508F3FC9F0809315056D
:10B7A0009091CA0740911305CACF80911805815026
:10B7B0008F3F01F1809318059091C80720911605DD
:10B7C000A5CF81E06DCFB1E0B093110584CF50914A
:10B7D00023085150509315058091BE038130E9F044
:10B7E00086958093BE039091CA07492F48234093C2
:10B7F0001305A7CF40910E08415040931805809142
:10B80000BF03813061F086958093BF039091C80794
:10B81000292F2823209316057BCF80E8E2CF80E8EC
:10B82000F3CFCF9108952FB7F8944FE150E05093A4
:10B83000CD004093CC0038E93093C90086E0809376
:10B84000CA008091CE005091C8005523D4F360EC1B
:10B850006093C8002FBF21E435E03F932F931F92E0
:10B860000E94990E0F900F900F900895EF92FF9203
:10B870000F931F93CF93DF93CDB7DEB722970FB609
:10B88000F894DEBF0FBECDBF482F4F5FCB0183536F
:10B890009B4268E170E00E943460E42EFF24F701CF
:10B8A000EE0DFF1DEA59F84F808191819C01220F16
:10B8B000331F280F391F260F371F37FD61C03595FD
:10B8C0002795359527953A832983DB0111960981C0
:10B8D0001A81A017B10794F589819A8101979A83FB
:10B8E0008983109145041936A0F187010E0D1F1DA3
:10B8F000F801EA59F84FA981BA8180819181A81B8A
:10B90000B90BCD0163E070E00E9434609B01660FCB
:10B91000771F620F731F0458184FF80171836083FB
:10B92000EE0CFF1C06E617E0E00EF11E69817A813D
:10B93000F70171836083443031F51FC0615070405E
:10B9400089819A818617970764F689819A81019681
:10B95000C6CFF701EE0DFF1DE458F84F118210829B
:10B96000EE0CFF1C06E617E0E00EF11E69817A81FD
:10B97000F70171836083443031F410927F0303C078
:10B980002D5F3F4F9CCF22960FB6F894DEBF0FBEBF
:10B99000CDBFDF91CF911F910F91FF90EF90089550
:10B9A000CF9380919F088F3149F080919F0899270C
:10B9B000807F9070409709F047C022C04091A00856
:10B9C00040931A053091A20830931C0590911C05F4
:10B9D00084ED989FC0011124880F892F881F990B2F
:10B9E000919580934504809145042091A30820936C
:10B9F0001B0580919F089927807F9070409721F5C3
:10BA0000C0919F08CF70CA30F8F49091A00890932D
:10BA100022057091A108709321056091A20860939E
:10BA200024055091A308509323056091210570913E
:10BA300022058C2F0E94365C6091230570912405AD
:10BA40008C2F8F5F0E94365CCF9108951F93CF9308
:10BA5000C82F8F3FC1F1109120051123C9F090919B
:10BA60001D05209120059217E0F480911E05809518
:10BA70008F3F09F466C080931E0530911E05C317E1
:10BA800079F11092200510921E05C0931F0577C012
:10BA9000CF3111F194E090931D052091200592176C
:10BAA00020F310912005E12FFF27E156F74FC083C7
:10BAB00080911E058C0F80931E05F0912005FF5F7D
:10BAC000F0932005E2CF80911F058F3F21F6109261
:10BAD000200510921E0553C095E090931D05DDCF03
:10BAE00040919F084F3179F180919F089927807F7D
:10BAF0009070409731F610919F081F701A3008F02F
:10BB0000C0CFE091A008E0932205B091A108B093C6
:10BB10002105A091A208A09324059091A3089093D9
:10BB200023056091210570912205812F0E94365CCA
:10BB30006091230570912405812F8F5F0E94365CF0
:10BB4000A0CF8EEF98CF7091A00870931A056091E6
:10BB5000A20860931C0590911C0584ED989FC0017C
:10BB60001124880F892F881F990B91958093450484
:10BB7000809145045091A30850931B05B5CFCF91F8
:10BB80001F9108951F920F920FB60F9211241F93C9
:10BB90002F933F934F935F936F937F938F939F93D5
:10BBA000AF93BF93CF93EF93FF93C091CE00CF3F5E
:10BBB000C1F1109120051123C9F090911D0520912C
:10BBC00020059217E0F480911E0580958F3F09F4BF
:10BBD00066C080931E0530911E05C31779F110923F
:10BBE000200510921E05C0931F0577C0CF3111F1BB
:10BBF00094E090931D0520912005921720F3109159
:10BC00002005E12FFF27E156F74FC08380911E05E5
:10BC10008C0F80931E05F0912005FF5FF0932005A7
:10BC2000E2CF80911F058F3F21F6109220051092E0
:10BC30001E0553C095E090931D05DDCF40919F08F0
:10BC40004F3179F180919F089927807F90704097BC
:10BC500031F610919F081F701A3008F0C0CFE091A4
:10BC6000A008E0932205B091A108B0932105A0910E
:10BC7000A208A09324059091A308909323056091B6
:10BC8000210570912205812F0E94365C6091230569
:10BC900070912405812F8F5F0E94365CA0CF8EEFBC
:10BCA00098CF7091A00870931A056091A2086093D4
:10BCB0001C0590911C0584ED989FC0011124880FEC
:10BCC000892F881F990B9195809345048091450495
:10BCD0005091A30850931B05B5CFFF91EF91CF91E1
:10BCE000BF91AF919F918F917F916F915F914F9194
:10BCF0003F912F911F910F900FBE0F901F9018959D
:10BD0000FC014150504030F001900616D1F73197B8
:10BD1000CF0108958827992708955058192EEFD0FC
:10BD200001D0D2C0BA176207730784079507B1F133
:10BD300088F40EF410940B2EBA2FA02D062E622F2D
:10BD4000202D072E732F302D082E842F402D092EE5
:10BD5000952F502DFF275523B9F0591B49F0573E19
:10BD600098F0469537952795A795F0405395C9F7D4
:10BD700076F0BA0F621F731F841F30F48795779592
:10BD80006795B795F040939517FA0F2E0895BF1B4E
:10BD9000BB27BA0B620B730B840BF6CFDEF6DBC04E
:10BDA000AED001D091C0552359F0992369F09F5727
:10BDB0005F57951B33F442F4903811F4915805C045
:10BDC0009BC091589F3F09F4C6C0BB27112462173E
:10BDD0007307840730F4660F771F881FBB1F9150CD
:10BDE00098F311D00F920FD00F920DD0A0E8261724
:10BDF000370748071B0609F0A048BA2F602D7F912E
:10BE00008F9100240895A0E8002462177307840727
:10BE1000B10528F0621B730B840BB1090A2A660F67
:10BE2000771F881FBB1FA69581F7089597FB73D0D6
:10BE30009F3738F0FEE9F91B982F872F762F6B2F4D
:10BE400005C086C09695879577956795F150D0F790
:10BE50003EF490958095709561957F4F8F4F9F4FE1
:10BE60000895E89403C097FB0EF4F3DFB62F672F15
:10BE7000782F892F9EE9002427C00ED05EF004C0E1
:10BE80000BD026F001C008D019F020F48FEF0895F0
:10BE900080E0089581E0089597FB092E052600F8BB
:10BEA000689430D0E89407FC07C0621773078407D2
:10BEB000950721F008F400940794989408959A95B2
:10BEC000BB0F661F771F881F11249923A1F08823B9
:10BED000B2F79F3F59F0BB0F48F421F4002011F452
:10BEE00060FF04C06F5F7F4F8F4F9F4F881F9795F4
:10BEF000879597F908952CC09FEF80EC0895052E43
:10BF0000092607FA440F551F5F3F79F0AA27A517A6
:10BF100008F051E04795880F991F9F3F31F0BB27EC
:10BF2000B91708F091E0879508959F919F9111248A
:10BF3000E3CF97FB880F991F9F3F31F0BB27B917BD
:10BF400008F091E0879508959F919F911124D4CF97
:10BF500066277727882799270895D1DF01D0B4CFA6
:10BF6000992339F0552329F09F575F57950F13F404
:10BF70009AF1F1CF91589F3FE1F3629FA12D0F926B
:10BF8000BB27639FA00DB11DEE27729FA00DB11DB1
:10BF9000EE1FAF93AA27649FB00DE11D739FB00DF4
:10BFA000E11DAA1F6627829FB00DE11DA61F552720
:10BFB000749FE00DA11D551F839FE00DA11D561F0D
:10BFC000849FA00D511D852F7A2F6E2F1F900F90EB
:10BFD00088231AF4939539F48FCF000C111CBB1FE2
:10BFE000661F771F881F01280895629FD001739FE5
:10BFF000F001829FE00DF11D649FE00DF11D929F05
:10C00000F00D839FF00D749FF00D659FF00D992743
:10C01000729FB00DE11DF91F639FB00DE11DF91F67
:10C02000BD01CF0111240895991B79E004C0991F27
:10C03000961708F0961B881F7A95C9F78095089582
:10C04000AA1BBB1B51E107C0AA1FBB1FA617B7073E
:10C0500010F0A61BB70B881F991F5A95A9F780955A
:10C060009095BC01CD01089597FB092E07260AD0B3
:10C0700077FD04D0E5DF06D000201AF470956195B5
:10C080007F4F0895F6F7909581959F4F0895A1E20F
:10C090001A2EAA1BBB1BFD010DC0AA1FBB1FEE1F42
:10C0A000FF1FA217B307E407F50720F0A21BB30B8D
:10C0B000E40BF50B661F771F881F991F1A9469F709
:10C0C00060957095809590959B01AC01BD01CF0165
:10C0D000089597FB092E05260ED057FD04D0D7DF13
:10C0E0000AD0001C38F450954095309521953F4F6B
:10C0F0004F4F5F4F0895F6F7909580957095619535
:10C100007F4F8F4F9F4F0895F999FECFB2BDA1BDCC
:10C11000F89A119600B40895F7DF01921A94E1F7A6
:10C120000895F999FECFB2BDA1BD00BC11960FB61E
:10C13000F894FA9AF99A0FBE08950190F2DF1A94D2
:04C14000E1F7089586
:10C14400010A0144534C0050504D00496E74656718
:10C1540072616C4E69636B20202020496E746567A0
:10C1640072616C526F6C6C202020204163634E69B5
:10C17400636B202020202020202020416363526F05
:10C184006C6C2020202020202020204779726F47CB
:10C194006965722020202020202020486F65686572
:10C1A4006E576572742020202020204163635A203A
:10C1B40020202020202020202020204761732020C0
:10C1C40020202020202020202020204B6F6D706113
:10C1D400737356616C7565202020205370616E6EF8
:10C1E400756E672020202020202020456D70666118
:10C1F4006E67202020202020202020457273617447
:10C204007A6B6F6D706173732020204D6F746F7241
:10C214005F566F726E6520202020204D6F746F7200
:10C224005F48696E74656E202020204D6F746F72B4
:10C234005F4C696E6B7320202020204D6F746F72E9
:10C244005F52656368747320202020202020202002
:10C254002020202020202020202020446973746185
:10C264006E636520202020202020204F73644261CB
:10C2740072202020202020202020204D4B334D618F
:10C28400672043616C537461746520536572766FE3
:10C2940020202020202020202020204E69636B2095
:10C2A4002020202020202020202020526F6C6C2071
:10C2B400202020202020202020202020202020207A
:10C2C40020202020202020202020204A3136202019
:10C2D40020202020202020202020204A3137202008
:10C2E400202020202020202020202020202020204A
:10C2F40020202020202020202020204B616C6D61F4
:10C304006E5F4D617844726966742020202020207D
:10C3140020202020202020202020204B616C6D61D3
:10C324006E204B20202020202020204750535F4E99
:10C3340069636B20202020202020204750535F5227
:10C344006F6C6C2020202020202020C8000164FF76
:10C3540001FFFF280001806400737373FF03007DF5
:10C36400000064000B48616C6C6F2057656C7400AE
:10C3740000000000000000000000000000000000B9
:10C3840000000000000000000000000000000000A9
:10C394000000000000000000000000000000000099
:10C3A4000000000000000000000000000000000089
:10C3B40000000000000102030405060708090A0141
:10C3C400ECFF6446640A029696403A10FB3017B7B5
:10C3D400D13890D0030090D00300F401640053706E
:10C3E4006F727400004E6F726D616C00004265677D
:10C3F400696E6E65720000640A0B0D0B0C0E010170
:00000001FF
